:020000040800F2
:10500000D81B0020D9500008A18C00087D8300081F
:105010000000000000000000000000000000000090
:10502000000000000000000000000000399A0008A5
:105030000000000000000000E9920008519B0008F9
:10504000EB500008EB500008EB500008EB50000854
:10505000EB500008915D0008EB500008EB50000891
:1050600000000000EB500008B95C0008EB5000089D
:10507000EB5000089188000800000000EB50000889
:1050800000000000EB5000080000000000000000DD
:10509000EB50000800000000EB500008EB50000847
:1050A000EB500008EB500008EB500008FDA500088D
:1050B000EB500008EB50000800000000000000006A
:1050C0000448854600F044FD004800477DB90008CB
:1050D000C046C046D81B002004488047044800470B
:1050E000FEE7FEE7FEE7FEE7FEE7FEE7ED9B0008D2
:1050F000C150000830B50B46014600202022012493
:1051000009E00D46D5409D4205D31D469540491BFB
:105110002546954040191546521E002DF1DC30BD44
:10512000F0B51FB40646002082B005464024019128
:1051300000901BE0019922460F46304600F0F2FB3A
:10514000049A059B801A994110D3104619462246AD
:1051500000F0D8FB361A8F4101972246012000212A
:10516000009F00F0CFFB38184D4100902046641E90
:105170000028DFDC019B00982946324607B0F0BDCD
:1051800003460B439B0703D009E008C9121F08C060
:10519000042AFAD203E00B780370401C491C521E0B
:1051A000F9D27047D2B201E00270401C491EFBD216
:1051B00070470022F6E710B513460A460446194622
:1051C000FFF7F0FF204610BD30B50446002003462F
:1051D00000E05B1C934203D2E05CCD5C401BF8D046
:1051E00030BDF8B502464A40D40F42004B00520889
:1051F0005B089A4202D20246084611464A0023D072
:10520000C30D4A00DDB2120EAD1A202D35DA490267
:105210000126490AF6058A19002C00D052422021A5
:105220004F1B1146B9402A411018C20D9A4221D095
:10523000002C17D0012D08DCDA05801AD20F801956
:10524000D207DBB200F09AFBF8BDDA05801A012321
:1052500040001B06C01880185A428018CA0F10431D
:10526000490007E04908C2071143DA05801A80198E
:105270004008801800F07AFBF8BD61000122511A45
:10528000001BF7E70122D2075140AAE70122D2070B
:105290005040A6E7024670B54A40D30FDB074000F6
:1052A0002DD04A002AD0010E140E00021202091954
:1052B000400A520A8418E50104465443000A120ABF
:1052C0002E045043A4194219200CC543AA18120CED
:1052D0000125AD03521C521912047F39240400D059
:1052E000521C104301D44000491EC2B20C06C00932
:1052F0002018401C4008802A02D003E0002070BD26
:1053000040084000002900DA0020184370BD70B545
:1053100002464A40D50F40004A00ED0740085208B7
:10532000002814D0002A12D0C40DD30D4102012050
:10533000C0055202490A520AE41A091812187D34AB
:10534000914201D3641C00E04900002C01DA0020E6
:1053500070BD0023914201D3891A034340084900DC
:105360000028F7D100290AD0914202D10121C907B2
:1053700005E0914201D2012101E00121C943E0058C
:10538000C018401900F0F2FA70BD420005D042008A
:10539000120E52428A4201DB00207047C9050818EC
:1053A00070470000F0B507460846584087B0C00F68
:1053B000049048000E46590040084908BC1A88412C
:1053C00005D2384631461E4617460B46024658005F
:1053D000400810434DD0300D039040055900400D5A
:1053E000490D0590401A0290402873DA18030121F4
:1053F000000B09050843019004980092002806D08C
:105400001146019A49420020904100910190029872
:1054100040210A1A0199009800F074FA05460C46DA
:105420006B4607CB00F08FFAC0197141039A0E0D3D
:105430000023D71756401A467A40164344D0049AA0
:10544000002A2DD0029A012A039A15DC1205C01AEF
:10545000914101263605001C7141D20F059ED207ED
:105460000093019202962A46234600F0CDFA07B037
:10547000F0BD38463146FAE71605234A0F46B21802
:10548000C01AB74101210905001C4F4100187F4196
:10549000114618187941E20F10436D19644113E069
:1054A000E2076D0815436408C2071443039A0126F6
:1054B0001205C01A91413605001C7141CE07400803
:1054C00030434908C01851412A46234600F08FFA5C
:1054D000CDE7FFE7049801224000C117121A00230C
:1054E0008B4104983146C417381AA141EEE730B415
:1054F0000124E407634030BC54E730B40124E407DE
:10550000614030BC4EE700000000E0FFF0B51FB482
:1055100088B00B990998002448400999C00F4900A8
:1055200049080991C0070B990090490049080B915F
:1055300009990898A64608431CD00B990A98084375
:1055400018D0099801244000420D4800410D0998E7
:1055500024050003000B204309900B980003000B67
:1055600020430B9050181C4940180022019014460B
:10557000104605E0002001460DB0F0BD032801DA19
:10558000034600E003239C46C11A0AAE0AE05F000E
:1055900008ADED5B4F00F75B7D430027AA187C4107
:1055A000491C5B1E6145F2DD410004AB5A522104E7
:1055B000120C0A43240C401C0828DFDB01980290DF
:1055C0000099704601910090059B049A07990698EE
:1055D00000F01AFAD0E700000DFCFFFFF0B50C4612
:1055E0005C4085B0E40FE40703944C000026640897
:1055F00059009446490802460296224321D0624649
:105600000A431ED06200570D4A000E032303550DB6
:10561000012402462C492405781B1B0B360B40182D
:1056200023432643614600901C46501AB44103D3DD
:105630000098401C009002E0921800985B410028FE
:1056400003DA0020014605B0F0BD00200121090564
:105650000746864611E064461D46141BB54106D335
:105660006546521BB341744607430C43A646CD071B
:1056700040084908284392185B4105460D43EAD18A
:105680001046184313D060461946504071400843F5
:1056900006D06046101AB34106D20122002306E06C
:1056A00000220123DB0702E00122D24353100098BD
:1056B00074460105381C6141029C039D0019694133
:1056C00000F095F9BFE70000FD03000070B54B0046
:1056D0005B0803430BD04B005C0D0026334665424C
:1056E000B341D417AD1AA34102DB0020014670BDBF
:1056F00012053018514170BDC217C10F504010B58E
:105700004018CA079623002100F038F910BD10B5E3
:1057100000229623114600F031F910BD0EB5C217D4
:10572000C10F5040CA0740180021054B0293019257
:1057300000910A460B4600F067F903B000BD000077
:10574000330400000EB505490291002100910A467C
:105750000B46019100F058F903B000BD330400007E
:10576000C20F410040020123400ADB05D207090EA7
:10577000C0187F2901DA00207047962903DC9623A0
:10578000591AC84001E096398840002AF4D04042B6
:105790007047410040020122400AD205090E8018DC
:1057A0007F2901DA00207047962903DC9622511ADE
:1057B000C8407047963988407047000070B5CD0FDB
:1057C0004A0009030123090B1B0519430B4BED0785
:1057D0000024520D9A4201DA002070BD074B343389
:1057E0009A4203DC9A1A00F09DF802E0044951182D
:1057F00088402C43F1D0404270BD0000FF03000000
:10580000CDFBFFFF4A0009030123090B1B051943C8
:10581000094B10B5520D9A4201DA002010BD064B1B
:1058200034339A4203DC9A1A00F07CF810BD034925
:105830005118884010BD0000FF030000CDFBFFFFA2
:10584000C20FD207400040080BD0C10D0723DB0177
:10585000C91840020905400A1143C2084007114314
:10586000704700200146704710B5002904DB012471
:10587000E40740428C412146002B04DB1C460123F7
:10588000DB075242A3418B4200D1824210BD00008F
:1058900010B5002904DB0124E40740428C41214675
:1058A000002B04DB1C460123DB075242A341994233
:1058B00000D1904210BD0000CB0FDB07490010B5AE
:1058C000490802460A4307D00A0D07240903E401E8
:1058D000090B121B002A01DC002010BDC900440F77
:1058E0000C43C100E018D205801800F03FF810BD4D
:1058F0000122D207002800DB101A002900DB511A10
:105900008142704710B5202A04DB0146203A9140BD
:10591000002010BD914020239C1A0346E340194308
:10592000904010BD10B5202A04DB0846203AD04034
:10593000002110BD0B46D340D0402024A21A914034
:105940000843194610BD10B5202A06DBCB170846C0
:10595000203A1041C1170B4306E00B461341D040DB
:105960002024A21A91400843194610BD002904DAE8
:10597000401C490001D140084000704770B4002429
:10598000050C05D11024000402D1002921D01124D6
:10599000050E01D100020834050F01D10001241DBC
:1059A000850F01D18000A41C002801DB4000641C8D
:1059B000002908D020252E1B0D46F540A14000D01F
:1059C00001212943084301061B1B000ADB1D02D5E8
:1059D000002070BC7047DB05181880180029F8DA21
:1059E000401C4900F5D170BC40084000704710B51C
:1059F000002B08DA0024401C614192185B411A43D5
:105A000001D14008400010BDF0B51FB482B005467A
:105A10000C0003D0084604F0ABFE02E004F0A8FE40
:105A200020300246009021462846FFF76BFF049B7A
:105A3000059A04460F4618431143084314D01846EC
:105A400010431BD0009840210A1A18460599FFF709
:105A500069FF05460E46009A05990498FFF752FF24
:105A6000084305D0012004E02046394607B0F0BDC8
:105A70000020C11705430E432C43374300990E986D
:105A80006305401A7905E40A00220C43FD0A0A3036
:105A900002D500200146E9E70105101969410C9C77
:105AA0000D9D00196941FFF7A2FFDFE7FEB5002356
:105AB0001A461B1A8A4103DB0020014603B0F0BDE1
:105AC0004A000D0301212D0B0905520D0D43D1078D
:105AD00002D100186D41521E5110FF31FF310131CA
:105AE000002704463E4638460097019102460121B0
:105AF00000200905FFF716FFC3197141F818324657
:105B000084468E464A4161462846611A904104D334
:105B10006046241A954176461F46241900986D4127
:105B2000401C00903428E1DDF91930467041091B12
:105B3000A84103D20022D243134601E000221346BB
:105B400001980105381C7141FFF751FFB6E70000CD
:105B5000064C0125064E05E0E36807CC2B430C3CC0
:105B600098471034B442F7D3FFF7AEFA70C8000874
:105B700090C8000870B58C180578401C6B075B0F47
:105B800001D10378401C2A1106D10278401C03E0A1
:105B900006780E70401C491C5B1EF9D12B0705D4FA
:105BA0000023521E0DD40B70491CFAE70378401CE9
:105BB000CB1A921C03E01D780D70491C5B1C521E11
:105BC000F9D5A142D8D3002070BD000038B50446F5
:105BD000064805490068FFF78DFA604300E0401E63
:105BE00000900028FBD138BD40420F007801002012
:105BF000F8B50446006881688907890F012902D138
:105C00000168C90722D18168114A10261140012577
:105C100000290ED18168294381600120FFF7D6FF5A
:105C200001F010F807460CE001F00CF8C01B0A2840
:105C300007D9606D30436065A06D2843A0650120E1
:105C4000F8BD20680068C043C007EDD10020F8BD52
:105C5000170000801FB50B4800900B4801900B48BF
:105C600002900B48039069460A4805F077F90A4A02
:105C700008481146083905F05FF800F057FA00208F
:105C800004B010BD79C6000855C60008B5C60008A6
:105C9000B3C60008840100201000002010B50023C6
:105CA0001A4603E0845CE3189BB2521C8A42F9D383
:105CB000D84380B210BD000010B5034800F07EFD4F
:105CC000024800F07BFD10BD741700202C17002047
:105CD00030B5446C1C252C400125A540046C656042
:105CE000046863608368102B036803D099600068C0
:105CF000C26030BD9A600068C16030BD14490120A7
:105D000048720A4602205E32507203203C3A5072BA
:105D100004200E3A50720F480D4B00780870223163
:105D20000870203108770C495A1C08785871497856
:105D30009971233318715971203318775977107579
:105D400051751A461E32107551751076517670478E
:105D5000DC110020270100204801002010B503F0CD
:105D600041FE202003F0EAFE012005F061FB002047
:105D700003F0E4FE044805F0FFF9044805F0AEFC2A
:105D8000002005F0E3FC10BDE80000208380000047
:105D9000F8B505200121000700F040FF0025174C51
:105DA000002800D06560164E0221304600F036FF14
:105DB00000281BD1012020701248808F00280ED0AF
:105DC0000127BF0200223946304600F034FF0A2086
:105DD00004F022FF01223946304600F02CFF0A4829
:105DE000656000880A21484308490880012000F0C6
:105DF0004DFE022000F04AFEF8BD000064010020C4
:105E000000040050DC0D0020340100204601002079
:105E10007047000010B5084900224A6107494B68E5
:105E20004C1523434B604B68082423434B60C00947
:105E3000C001026010BD0000BC170020002002401D
:105E40007FB500250C460646039500F0EFFDE009FE
:105E5000029003A901960095684600F07FFD002896
:105E600004D000F0B7FD002004B070BD00F0B2FD1A
:105E70000120F9E710B5002302E0C45CCC545B1CA0
:105E80009342FAD310BD000010B5214A0021906959
:105E9000C305204804D54169022319434161911586
:105EA00093699B0505D5436901242343436163023C
:105EB000194393695B0505D543690824234343616E
:105EC000E301194393691B0505D543690424234362
:105ED00043616302194393699B0405D54369102408
:105EE000234343616302194393699B0304D54469C7
:105EF00020231C43446119439369DB0305D543699F
:105F0000402423434361A0020143916110BD00007E
:105F100000200240BC17002070B5054600F092FE3C
:105F20000646184C0AE0681C08D0002D04D000F08A
:105F300089FE801BA84201D9032070BDA069C0075B
:105F4000F1D1A069800701D50220A061A069C00538
:105F500011D4A06980050ED4A06940050BD4A069B6
:105F6000000508D4A069800405D4A069800302D488
:105F7000A069C00303D5FFF787FF012070BD002093
:105F800070BD000000200240F8B517460026054607
:105F90000C4600F04BFD09E029460220226800F083
:105FA00027FD002804D1241D2D1D361DBE42F3D32C
:105FB00000F010FDBE4201D20020F8BD0120F8BD66
:105FC00010B5084902460020054B497905E0440018
:105FD0001C5B944203D0401CC0B28842F7D310BD72
:105FE000681300207000002010B500F01CFE10BDEA
:105FF00010B5094801F046F880B2FFF7A3FB074A45
:10600000074BFFF783FA0022064BFFF7E7FAFFF78B
:10601000F9FB80B210BD0000E0150020F853E3A5A5
:106020009B843E4000408F4070B53A493A4A002078
:106030008300401CC0B2D1501428F9D338493748E6
:106040000A7802754978417536490A7802764978A6
:10605000417632490520133148720A2005F02EFBA3
:106060007D20C00005F044FB2C49002213310C2098
:1060700005F00EFC00210C2005F01CFC022005F0B0
:106080006DFB274D284C203D00210F2005F096FA8E
:1060900020426863F8D0686B411C38D0400435D585
:1060A0008122D20100210F2005F0C7FB0021102022
:1060B00005F084FA41061848490E0022C43805F05C
:1060C000B3FA154CC43C607A05281FD10222154949
:1060D000601DFFF779F8002818D11148A67C6E7171
:1060E0000422611C3030FFF74BF82146133108467B
:1060F00072000C465130FFF743F8687921464200A0
:1061000005484838FFF73CF80320287070BD04F0BC
:10611000A3FB0000FFFF0100C81300203D12002078
:10612000900000204801002000D0272410B5144C16
:106130001448224610321146083904F0FDFD0022B1
:10614000114BE168A068FFF749FA104A104B05F0BF
:1061500023FD00220F4BFFF7D0F900220E4BFFF773
:10616000D5F9FFF7A9FB206000221346E168A0687B
:10617000FFF77AFB01D0206810BD0020206010BD21
:10618000000000208401002000AA8F406C45D9CC7B
:10619000955BC83F0000F03F40A5E54010B50848BA
:1061A00000F096FA0A21064800F032FA044800F09E
:1061B0001DF9800503D5024800F01AF980B210BD20
:1061C00084150020F8B52F4D00220121284600F04B
:1061D00032FDFFF7E3FFFFF79AFA2B4E3146FFF748
:1061E00096F82A4C0122A0601146284600F023FDB3
:1061F0002749A068002588423EDB2078254F0028EB
:1062000015D02570FFF7CAFFFFF781FA3146FFF777
:106210007EF8A060FFF714FB00223B46FFF767F90A
:1062200000221D4BFFF772F9FFF746FB6060A06884
:10623000FFF706FB00223B46FFF759F9174A184BB8
:10624000FFF764F906460F466068FFF7F9FA134A4C
:10625000144B5242FFF75AF932463B46FFF7A2F879
:10626000FFF72AFB10496060884201DD616004E0AD
:10627000FF21C905C84200D365606068FFF789FA4D
:10628000C0B2F8BD0004005000401B44480000208C
:106290000000604000000C4000E0644033333333C2
:1062A00033B33040CCCCEC3F0000C842F8B50546D3
:1062B00004464035287C0026012808D00120287497
:1062C000206881688907890F01290ED101E0022029
:1062D000F8BD0168C90708D0606D202108436065DA
:1062E0000126002028743046F8BD616DFF2201327E
:1062F0009143022211436165C1688907890F0091AA
:10630000C16889088900C1602068816892071143CB
:10631000816000F097FC07460EE000F093FCC01B84
:106320000A2809D9606D022188431021084360655D
:10633000002028740120F8BD206880680028ECDB6C
:106340002068C168009A1143C160606D80088000B8
:10635000401C6065C5E70000F8B506460D464036AE
:10636000317C01290DD00121317401688A685207FE
:1063700009D5416D20221143416500203074012070
:10638000F8BD0220F8BD174B6A68D80547109A423D
:10639000154C8A6A2B6812D05B035B0B1A438A6226
:1063A0002968490305D5A1680143A1600A20FFF7C8
:1063B0000DFC2868800312D5A06838430EE05B030B
:1063C0005B0B9A438A622968490302D5A16881431D
:1063D000A1602868800302D5A068B843A0600020AF
:1063E0003074F8BD0110000000270140406D704777
:1063F0000068006C7047000070B5040006D0606D46
:10640000264600254036002802D006E0012070BD57
:10641000A5653574204600F0D3F8606DC00603D43E
:1064200021688868400705D5606D102108436065C4
:106430003574EBE7606DFF22013290430222104376
:10644000606588688207920F5B48012A02D10A685A
:10645000D2072BD1032362689B079A4205D05B4287
:106460009A4202D05B009A4209D10A6992009208CE
:106470000A6121680A6963681A430A610CE00A69C3
:10648000920092080A6181680F2292049143816010
:1064900081686268114381602168CA6818239A4341
:1064A000CA602168CA68A3681A43CA608168012269
:1064B0005206914381608168A28E52061143816029
:1064C00020688168C90004D4816801221207114341
:1064D00081602068C168394A1140C1602069E16863
:1064E000022825D000200143204620300278037B7B
:1064F00052035B001A431143226B1143A2699203BA
:106500001143E269D20311432268D3681943D16071
:10651000616A0A46FF3AC23A05D0A26A114322686C
:10652000D3681943D16042780121012A02D00BE0DF
:106530000420D8E70078002823D0606D2022104383
:106540006065A06D0843A065E06B012820681FD03E
:106550000169C90703D00169490849000161206840
:106560004169C908C900416120684169A26B1143B2
:106570004161A565606D80088000401C6065002059
:1065800070BD2068C26801231B041A43C260DBE7A8
:106590000269FF239B009A43026120680269236C11
:1065A000A66C1A43636C33431A4302612068026984
:1065B0000A430261D3E70000002701401902FEFFF1
:1065C00010B586B0044614216846FEF7F2FD0E4968
:1065D0002068884216D10D48416B42151143416332
:1065E000C16A01221143C162C06A69461040059028
:1065F0000220009003200190002002900520000757
:1066000000F050FA06B010BD002401400010024016
:10661000F8B504464069254640350E4608280BD09B
:106620002068C068C00709D0606D202108436065FC
:10663000002028740120F8BD082700E00C2700F096
:1066400001FB009011E0701C0FD0002E05D000F06F
:10665000F9FA0099401AB04207D9606D0421084345
:106660006065002028740320F8BD20680068384267
:10667000E9D0606D01214902084360652068C16866
:1066800009058A0F0C21002A1BD12022125D002A45
:1066900017D10268120714D5826853070122002B14
:1066A00008DB43688B434360606D130298431043DB
:1066B000606506E0606D202318436065A06D10439F
:1066C000A065A069002801D1206801600020F8BD04
:1066D00070B50446216800208968490721D4254601
:1066E0004035297C01291CD001212974E169012947
:1066F00004D02046FFF77CFA002811D1616D0A4AC8
:106700001140FF220132114361650021A165297406
:1067100022681C21116021688A6804231A438A6058
:1067200070BD022070BD0000FEF1FFFF30B50146D4
:1067300020314A790023022A04D00422C2630B715B
:10674000012030BD026814680E25AC431460026855
:106750001468640864001460446C1C221440012214
:106760001546006CA54045604A7118460B7130BD56
:1067700070B50024014620314A79022A03D0042151
:10678000C163012418E0026813680E25AB4313604F
:10679000026813685B085B001360436C1C221340A3
:1067A000012215469D40036C5D604A7100220A710A
:1067B000816B002900D08847204670BDF0B4016C81
:1067C0000D6801680C68466C1C2304221E401746A5
:1067D000B7402F420ED067070CD50C68A40602D430
:1067E0000C6894430C60416C19408A40016C4A600B
:1067F000016B1AE00227B74002462F402032002FDB
:1068000017D0A70715D50C68A40605D40C680A256F
:10681000AC430C6001215171446C02211C40036C9B
:10682000A140596000211171C16A002918D0F0BC43
:1068300008470827B7402F4212D0240710D50C680C
:106840000E25AC430C60446C01211C400B46A34058
:10685000046C6360C163517100211171416BE4E705
:10686000F0BC704770B504003CD01F482568142167
:106870002818FEF73FFC800060641C482064022159
:10688000204620300246417129681948E3680140DA
:10689000A06866691843236933431843A369184302
:1068A000E3691843236A1843084328600121A0685C
:1068B0008903884210D00D488030836A656C1C21A2
:1068C0000D400F26AE40B3438362656C63680D4094
:1068D000816AAB400B4383620020E0630121517168
:1068E000107170BD012070BDF8FFFDBF00000240B7
:1068F0000F80FFFFF8B504468C4620300179002553
:10690000012909D00126067141790027012905D006
:10691000077102252846F8BD0220F8BD0221417109
:10692000E763206801684908490001606146204624
:10693000FFF7CEF9206B00282068016801D00E22F5
:1069400005E0042291430160206801680A22114396
:1069500001602068016831430160DBE7F8B51A4E39
:106960000546307C0F46012807D0012030741748B7
:10697000FFF7D2FA010002D021E00220F8BD00208A
:10698000C04338606C6814E02046FFF743FA0F48B4
:10699000FFF7C2FA01460E48426808239A43426054
:1069A000426843159A434260002901D03C6006E0EA
:1069B0008034A8686A68C0018018A042E4D800202A
:1069C00030740846F8BD0000BC17002050C300001A
:1069D000002002400548416802221143416041689D
:1069E0000122114341600020704700000020024056
:1069F000F8B50C4C1646207C0F46012808D0012023
:106A000020740948FFF788FA0025002802D006E024
:106A10000220F8BD65613E600348FFF77DFA2574EA
:106A2000F8BD0000BC17002050C3000011484168A9
:106A3000C9070BD0EFF3108172B60F4AC2600F4A3C
:106A4000C26081F310884168C9070ED14168890787
:106A50000DD5EFF3108172B6094A0261094A02614D
:106A600081F310884068800701D50120704700201D
:106A70007047000000200240EFCDAB8905040302FF
:106A8000BFAE9D8C161514137047000010B5044955
:106A90004A69024202D04861FFF7F6FF10BD0000CC
:106AA00000040140FCB500230124A2E027462A4649
:106AB0009F403A406FD04D68012D05D0022D03D084
:106AC000112D01D0122D16D185680326AC465D002C
:106AD000AE46AE406546B543AC46CE687546AE4060
:106AE00065462E43866046680D79BE43ED06ED0F80
:106AF0009D4035434560C6685F000325BD40AE46F6
:106B0000AE4335468E68BE402E43C6604E68022EA8
:106B100001D0122E14D1DE08B60036180196366A5E
:106B20005D07B446EE0E0F25B54000966646AE43AF
:106B3000B4460D69009EB54066462E43019D2E6207
:106B400006687546AE430D79AD07AD0FBD403543C0
:106B500005604D68ED004BD5294D6E6B26436E6385
:106B60009E08284DB6007519AC46AD689E07360FD5
:106B70000F27B740BD4305273F07B84201D1002783
:106B800015E0214FB84201D1012710E01F4FB84254
:106B900002D102270BE02BE01D4FB84201D10327A1
:106BA00005E01C4FB84201D1052700E00627B74099
:106BB0002F436546AF60184D2E684F689643FF031C
:106BC00000D516432E606E684F689643BF0300D50C
:106BD00016436E60AE684F689643FF0200D51643B9
:106BE000AE60EE684F689643BF0200D51643EE6074
:106BF0005B1C0A681546DA4000D057E7FCBD000070
:106C00000010024000000140000400500008005045
:106C1000000C0050001C00500004014000690840B6
:106C200000D001207047426913460B401B0491437A
:106C30000B4383617047002A01D0816170478162F4
:106C40007047000001488068704700006C01002018
:106C50000248816802788918816070476C010020C1
:106C600010B5084800240168402211430160204605
:106C700000F00AF8002801D0012401E000F04CFAED
:106C8000204610BD0020024070B504460D4D7D2009
:106C90002978C000FEF72EFA01460B480068FEF77F
:106CA00029FA00F035FF002809D1042C07D2002270
:106CB0002146401E00F058FA00206C6070BD012093
:106CC00070BD00006C010020780100207047704703
:106CD000F8B5654CA078401CA07001202071A08BF5
:106CE000401CA0836148008802F0E4FE208AFEF781
:106CF0000EFD01467F20C005FEF709FB5C4D0646F0
:106D00002968FEF76EFA28600120A16AC005814259
:106D100001DA084603E03046FEF7B8FAA062FF2128
:106D2000C9050025C84200D3A562607800280BD1B0
:106D300002215048FFF772FF02004F494F4817D019
:106D40000022FFF778FFA56302214A48FFF766FF9C
:106D50004B4E002855D0A563B08AFEF7D8FC444FAF
:106D60003968FEF7C5FD5FD24649012008705DE035
:106D70000122D1034148FFF75EFF208AFEF7C7FCDE
:106D800001467F20C005FEF7C2FAA16BFEF729FA83
:106D90003D49A0638842D7DD39480127F9264030B4
:106DA00000900A213046FEF7A5F9002903D13249A7
:106DB0003248FFF719F902212E48FFF72FFF00286C
:106DC00001D0002701E0002F12D102212948FFF74E
:106DD00025FF00280CD104F0A7FE0099012088802F
:106DE00005F0FEFB642003F017FF29492748C8601F
:106DF0000A2003F011FF3046761EF6B20028D0D1EB
:106E0000A2E7208AFEF783FC01467F20C005FEF73B
:106E10007EFAA16BFEF7E5F91E49A06388429BDB71
:106E20001B491A48C86097E716480570708F401EC6
:106E3000FEF762FC3968FEF75BFD06D86079002832
:106E400003D015490120087001E013480570708FC8
:106E5000FEF75DFC3968FEF74BFD04D2607900282F
:106E600001D004F025FEF8BD240100208E00002092
:106E70006801002000040050008000000000005065
:106E8000DC0D002076000020000040400400FA05E0
:106E900000ED00E00000A04084000020704770B5C5
:106EA000040010D0022025462035A873204601F0AA
:106EB000F7FCA87B032805D0204600F0B9F8002095
:106EC000A873687370BD012070BD7047704710B51E
:106ED000044600680168C943C90708D18168C943ED
:106EE000C90704D1012141602046FFF7F1FE206867
:106EF0000168C943890708D48168C943890704D454
:106F0000022141602046FFF7E1FE20680168C94385
:106F1000490708D48168C943490704D40421416062
:106F2000204600F0F7F820680168C943090708D433
:106F30008168C943090704D4082141602046FFF74E
:106F4000ADFF20680168C943C90608D48168C943F8
:106F5000C90604D4102141602046FFF7B8FE20681E
:106F60000168C943890608D48168C943890604D4E5
:106F7000202141602046FFF7A9FF20680168C9432E
:106F8000490608D48168C943490604D440214160B8
:106F90002046FFF79AFF10BDF8B5040005D025463E
:106FA0002035A87B002802D006E00120F8BD002093
:106FB0006873204600F04EF80220A8732068C2686B
:106FC00084466368012B01D106208243164861691B
:106FD000814202D0072040038243002B01D1D820F8
:106FE00082431248A668024018463043676A266A00
:106FF0003E433043A66A30431043002B02D0012B9E
:1070000004D005E02369E2691A4300E0E268104316
:10701000054A914202D0A269114308436146C86003
:107020000120A8730020F8BDFFFF0000F8F119FF50
:1070300010B500680549884207D10548816B4900B1
:10704000490881630D2000F073F810BD007C0040FA
:107050000010024010B50068084988420CD1084869
:10706000816BC20411438163002201210D2000F0D5
:107070007BF80D2000F06CF810BD0000007C004093
:10708000001002400068C06970470000F8B504466F
:107090000220254620351746A8731D480268C30400
:1070A0001A4302602068C2689B121A43C2602068BB
:1070B0000269012632430261226810205060206874
:1070C00081611021204601F05BFC03281FD021685C
:1070D00008204860206847610821204601F050FCE4
:1070E000032814D0204601F0DBFBA87B03280ED038
:1070F0002068816831438160206801693143016102
:1071000020680169042211430161AE730020F8BDBB
:1071100000040140704700000448416B0122114304
:107120004163816B02041143816370470010024088
:10713000002809DBC106C90E012088400349086008
:10714000BFF34F8FBFF36F8F7047000080E100E007
:10715000002805DBC106C90E0120884001490860EE
:107160007047000000E100E010B503F053FB10BDD4
:1071700002494A6882434A6070470000007000403C
:107180000248016882151143016070470070004099
:1071900002494A6802434A6070470000007000409C
:1071A0000548016802221143016004480169042274
:1071B0001143016130BF70470070004000ED00E0F6
:1071C000F0B5154A1368154D54152D6A2340ED0787
:1071D000ED0F002B04D0002D02D01668A6431660D8
:1071E0001668B608B600064316600D4807690426FF
:1071F0003743076101290DD040BF20BF20BF01697F
:10720000B1430161002B04D0002D02D0106820434F
:107210001060F0BD30BFF2E7007000400000014098
:1072200000ED00E0F8B5044600780027534D8006D5
:1072300071D5524E403EB06BC00004D4B06BA9056E
:107240000843B06301274E480168C90511D401689D
:10725000821511430160FFF7F5FC009005E0FFF790
:10726000F1FC0099401A642837D845480068C005E9
:10727000F5D532680321090560680A400140914252
:1072800008D08103890F032904D13168890301D50E
:107290000120F8BD2A69032109040A4022D00840D0
:1072A00090421FD0207880061CD528692A6988431F
:1072B0000121C9040A432A612A698A432A61286193
:1072C000C0050FD5FFF7BEFC009008E0FFF7BAFC41
:1072D0000099411A2B48814201D90320F8BD286941
:1072E0008005F3D561688803800F032805D13268D3
:1072F0000005824301400A43326028690322616825
:107300001204114008432861002F04D0B16B012002
:1073100000078143B1632078C00705D0E868A16801
:10732000800880000843E8602078800705D5E86879
:107330000C218843E1680843E8602078400706D5BF
:10734000E86803218902884321690843E8602078BE
:10735000000706D5E86803210903884361690843EB
:10736000E8602078000606D5E86803218904884390
:10737000A1690843E8600020F8BD00004010024009
:107380000070004088130000F8B50E46050038D0A4
:107390005E480068C007C00FB04214D25B4C206842
:1073A0004008400030432060FFF74CFC074605E0F2
:1073B000FFF748FCC11B564881427AD82068C007B5
:1073C000C00FB042F4D12878524C800705D5E06850
:1073D000F0218843A9680843E0602878C00752D0AC
:1073E0006868022806D0032807D0216801280AD03F
:1073F000890504E02168890301E0216889010029E9
:1074000003DB0120F8BD4907F9E7E1688908890035
:107410000143E160FFF716FC0746686802280AD0BE
:10742000032814D001281ED029E0FFF70BFCC11B54
:10743000374881423DD8E0680007800F0228F4D128
:1074400021E0FFF7FFFBC11B3148814231D8E068E2
:107450000007800F0328F4D115E0FFF7F3FBC11BF1
:107460002B48814225D8E0680007800F0128F4D11D
:1074700009E0FFF7E7FBC11B2548814219D8E06806
:107480000007800FF5D121480168C907C90FB14233
:1074900017D901684908490031430160FFF7D2FB61
:1074A000074608E005E0FFF7CDFBC11B1848814205
:1074B00001D90320F8BD15480068C007C00FB042CD
:1074C000F1D12878400706D5E068072109028843F2
:1074D000E9680843E0602878000707D5E0680721DD
:1074E000C90288432969C9000843E06000F03AF8FE
:1074F000E168094A0906090F515CC840074908605C
:1075000007480068FFF7C0FBF8BD000000200240FC
:107510008813000000100240BAC70008780100205C
:1075200070010020044805490068C968044A4905FB
:10753000490F515CC840704778010020001002409C
:10754000D3C70008044805490068C968044A89048B
:10755000490F515CC840704778010020001002407C
:10756000D3C7000870B51A4AD3681A490C201840CE
:107570008D0004280CD04E00082810D00C2810D004
:1075800050680004410F0120C003491C884070BDB1
:107590001068C00601D5084670BD284670BD30464B
:1075A00070BD98020C4C000F205C1B029C0FD3682E
:1075B000641CDB0301D5314603E01268D20600D417
:1075C000294603F0ECF822460023FDF7A9FD70BD23
:1075D0000010024000093D00CAC70008FEB50500C2
:1075E0007ED0FE4CE7680C20E668074001200004CE
:1075F00006402878C00747D0082F05D00C2F0AD1A5
:1076000001200004864206D1206880033CD56868CA
:107610000028E5D038E0012069680004814203D1E8
:1076200021680143216011E0052301221B0492041B
:107630009942216802D111432160F1E78143216021
:10764000216801400091206890432060686800280C
:107650000DD0FFF7F7FA009005E0FFF7F3FA009975
:10766000401A64287BD820688003F6D50CE0FFF729
:10767000E9FA009005E0FFF7E5FA0099401A64285E
:10768000F0D820688003F6D42878800756D50923DF
:10769000E868042F0DD00C2F01D1002E09D000284E
:1076A0003CD02168994301432160FFF7CBFA06469D
:1076B00028E02168490701D5002891D061681F2280
:1076C000120291432A6912021143616021689943B1
:1076D00001432160FFF746FFE16809060A0F00E059
:1076E0008BE1BF49895CC840BE490860BE4800685C
:1076F000FFF7CAFA002873D120E0FFF7A3FA801B36
:107700000228AFD820684007F7D560681F2109021A
:10771000884329690902084360600FE02068400837
:1077200040002060FFF78EFA064604E0FFF78AFA71
:10773000801B022896D820684007F7D42878C00616
:1077400060D5002F0CD0A86900284AD02068FF21FE
:10775000013108432060FFF775FA06462EE0C1E0CC
:107760002068800502D5A8690028A6D06068072196
:1077700049038843296A084360606068297F0002E2
:10778000000A090608436060286A410B0120C00313
:10779000491C8840E16809060A0F9149895CC84084
:1077A0009049086090480068FFF76EFA002817D1EA
:1077B00028E0FFF747FA801B0228A2D8206880053E
:1077C000F7D56068072149038843296A0843606048
:1077D0006068297F0002000A09060843606011E022
:1077E000E2E02168FF20013081432160FFF72AFA9F
:1077F000064604E0FFF726FA801B022872D82068AC
:107800008005F7D42878794E000724D568690028C8
:10781000306910D0012108433061FFF713FA00905E
:1078200005E0FFF70FFA0099401A02285AD830698C
:107830008007F6D50FE0400840003061FFF702FAFC
:10784000009005E0FFF7FEF90099401A022849D898
:1078500030698007F6D42878400766D5002002906A
:10786000A06BC00006D4A06B012109070843A063E8
:10787000012002905E480168C90511D40168821593
:1078800011430160FFF7DEF9009005E0FFF7DAF938
:107890000099401A642825D855480068C005F5D5D8
:1078A000FF20AA680130824203D13169014331616E
:1078B00011E001218902002A07D005231B029A4208
:1078C00003D132690A433261EFE7326982433261A0
:1078D000306988433061A868002810D0FFF7B2F9FA
:1078E000009008E05FE0FFF7ADF901460098091A43
:1078F0004048814257D830698005F4D50DE0FFF744
:10790000A1F9009006E0FFF79DF90099411A394866
:10791000814248D830698005F5D40298002804D007
:10792000A06B012109078843A063686A002866D01C
:107930000C2F3ED0012636060228206805D0B04321
:107940002060FFF77FF905462FE0B0432060FFF786
:1079500079F9074604E0FFF775F9C01B022822D821
:1079600020688001F7D4E96AA86AE2680843296BB5
:10797000FD231B049A4311430843E0602068304311
:107980002060FFF75FF9054604E0FFF75BF9401B55
:10799000022808D820688001F7D530E0FFF752F9B7
:1079A000401B022801D90320FEBD20688001F5D4C8
:1079B00025E00128F8D0E06801210904AA6A014005
:1079C00091421AD10F218904EA6A0140914214D1EF
:1079D000032189050840296B88420DE00010024010
:1079E000BAC7000878010020700100204010024052
:1079F000007000408813000001D00120FEBD00206F
:107A0000FEBDF8B504000ED0FF27606A05370025DB
:107A100000280AD02561656126464036A562707C43
:107A2000002807D00AE00120F8BD6068B842F3D012
:107A3000E561F1E73574204600F03EF802217174EB
:107A40002068026840239A4302602123A26860688C
:107A50009B021A4038401043E3688A0213401843DF
:107A600023690B40217D1843C907C90F0843A16949
:107A7000931019400843E169382319400843216AEB
:107A8000802319400843A16A9300194008432168E4
:107A90000860A0690421000C0840616A10231940A5
:107AA0000843216848602068C1699143C1616565E8
:107AB000012070740020F8BD10B586B00446142172
:107AC0006846FDF776FB10492068884219D10F48B7
:107AD000416B821411434163C16A01221143C162A7
:107AE000C06A002110400590E02000900220019023
:107AF0000320039002910491052069460007FEF7D8
:107B0000D1FF06B010BD000000300140001002405F
:107B1000094910B5401E884201D9012010BD074C0B
:107B200060610321081F02F075FE0020A06107209C
:107B30002061002010BD0000FFFFFF0000E000E01A
:107B4000F0B502462032137E012B1ED0012515769A
:107B50000223537606687468B3687027BC430F68C5
:107B6000274377600068AC07A04205D0084CA042CC
:107B700002D0084CA04204D180244968A343194391
:107B80008160557600201076F0BD0220F0BD000027
:107B9000000801400014014070B5050005D02C46D6
:107BA0002034607E002802D006E0012070BD002055
:107BB0002076284600F010F802206076291D2868FB
:107BC00002F040F80120A077A076E0762077607779
:107BD0006076002070BD000000680121890788429E
:107BE00004D10348816B0122114381637047000077
:107BF00000100240F8B5054604462035287E0128CD
:107C000017D001262E7602206876226890687727A2
:107C1000FF23B8431B02984390600A68502A31D072
:107C20000EDC202A4BD006DC002A48D0102A3AD19C
:107C300045E00220F8BD302A41D0402A33D136E059
:107C4000602A27D0702A12D001200003121A2AD0ED
:107C5000824228D1CB684A688968206802F02BF8F4
:107C60002068816801229203114381601BE0CB6888
:107C70004A688968206802F01EF8216888683843DD
:107C8000886010E0CA684968206802F08EF85021C8
:107C9000206806E0CA684968206802F097F8602109
:107CA000206802F013F86E7600202876F8BDCA68C6
:107CB0004968206802F079F840212068F1E7114610
:107CC0002068EEE710B586B0044614216846FDF73B
:107CD00070FA012120688907884212D10A49CA6ACC
:107CE00002200243CA62C96A019001400591410223
:107CF0000091002102910391049069460348FEF728
:107D0000D1FE06B010BD000000100240000400507B
:107D1000F8B5064604462036307E0D4601280BD0C5
:107D2000012008273076002A08D0042A16D0082A15
:107D30002AD00C2A4DD137E00220F8BD206801F08E
:107D4000CDFF2068816939438161206881690422FF
:107D50009143816120688169EA6812E0206801F03E
:107D6000D5FF206881690122D20211438161206818
:107D70008269012189028A43826120688169EA68F7
:107D800012021143816124E0206801F0D8FF2068CD
:107D9000C1693943C1612068C16904229143C1614D
:107DA0002068C169EA6812E0206801F0E3FF2068FA
:107DB000C1690122D2021143C1612068C269012157
:107DC00089028A43C2612068C169EA6812021143CC
:107DD000C16100203076F8BD70B5050005D02C4695
:107DE0002034607E002802D006E0012070BD002013
:107DF0002076284600F00FF802206076291D2868BA
:107E000001F020FF0120A077A076E0762077607750
:107E10006076002070BD704770B505462C46022084
:107E20002034002908D004290BD008290ED0627F05
:107E3000012A10D0012070BDA27E012AFAD1A076BD
:107E40000AE0E27E012AF5D1E07605E0227F012AF0
:107E5000F0D1207700E060770122286801F01EFF52
:107E60000122286892070121904205D0074A9042DA
:107E700002D0074A904204D182685207520F062A64
:107E800002D002680A430260002070BD0008014071
:107E90000014014070B504460D460068002201F050
:107EA000FDFE2068016A0C4A114203D101684908AD
:107EB0004900016001202034002D06D0042D06D099
:107EC000082D06D06077002070BDA076FBE7E07635
:107ED000F9E72077F7E700001111000070477047BD
:107EE00070470000F8B502680446D06911689668CA
:107EF000814B05461D402023002D6CD0F7077F4D98
:107F0000FF0FBC460D402F4379D02546C70780356B
:107F1000002F06D0CF0504D5012717622A683A43FF
:107F20002A60820708D5F20706D0276802223A6243
:107F30002A6804273A432A60420708D5F20706D088
:107F40002668042232622A68022632432A60020727
:107F50000AD50A461A406646324305D026680822EA
:107F600032622E6816432E60020508D54A0106D5F6
:107F700001222668D20232622A681A432A602A68DD
:107F8000002A30D0800606D5880604D5616E002907
:107F900001D020468847286821688968490602D4AC
:107FA0002821084225D0204602F03FF92068816848
:107FB000490619D5826840218A438260206F0028D3
:107FC00012D04F498163206FFEF7D2FB00280AD000
:107FD000206F816B06E0850611D58D060FD5616E89
:107FE00077E020468847F8BD2046FFF779FFF8BDC7
:107FF00005E02046FFF774FF00202860F7E7256EB4
:10800000012D56D1C50654D5CD0652D5102616627F
:108010002068816825464906403500292ADA226F02
:10802000116849680904090CE1D02F8B8F42DED911
:10803000698311680968890617D401683201914380
:108040000160206881684908490081602068816872
:10805000402291438160E367002020662068016828
:10806000B1430160206FFEF761FB288B698B401ADA
:1080700081B21AE0298B6A8B891A6A8B89B2002A2D
:10808000B5D00029B3D00268FF252135AA4302608C
:1080900020688268520852008260E36700202066F0
:1080A000606620680268B24302602046FFF716FF50
:1080B0009DE7C50208D5750206D5012000051062AE
:1080C0002046FFF70CFF92E7050605D50D0603D500
:1080D000A16E002985D18AE7400688D5480686D555
:1080E000116820464024A143116083670021816606
:1080F00000F043F97BE700000F08000020010004B6
:1081000051A1000810B5040003D0A06F002802D0D0
:1081100007E0012010BD002174200155204600F029
:1081200027F82420A06720680168490849000160F9
:10813000204602F0CDF80128ECD0606A002802D079
:10814000204601F0E5FE206841680922D2029143F1
:108150004160206881682A2291438160206801681B
:10816000012211430160204601F038FF10BD0000DC
:10817000F0B587B0064614216846FDF71AF82C4979
:108180003068884251D12B48416B01229203114340
:108190004163C16A01221143C162C06A00251040D7
:1081A00005900320400200900220032701A9A1C1ED
:1081B00004200490052069460007FEF773FC1F4C5D
:1081C0001D48A560E56081C48027E560A760202088
:1081D000256160610002A0611848083CFEF742FB7F
:1081E000002801D0FDF714FE3467A662144C124833
:1081F0002146143820600320606010200831A1C19E
:108200006561A561E56120462562FEF72BFB00282C
:1082100001D0FDF7FDFDF466002201211B20A662BE
:10822000FEF7A2FF1B20FEF793FF07B0F0BD000092
:108230000038014000100240300002402C1700209E
:108240007417002070B5C36F202B27D100290BD0E5
:10825000002A09D0012483682403A34206D10369BC
:10826000002B03D1CB0701D0012070BD0346603342
:108270001C7D012C12D001241C7500230366084CC0
:108280000368A34207D05C68240204D51C6801255A
:10829000AD062C431C6002F01BF970BD022070BDBE
:1082A0000048004070477047FFB50446806F83B0B8
:1082B00017460D4620285ED1002D0AD0002F08D089
:1082C000A168C001814207D12069002804D1E807D4
:1082D00002D0012007B0F0BD204660300090007D44
:1082E000012848D000980121017500208021085103
:1082F0002120A067FEF7A6FC264640360190378273
:1083000077820120A1680003814202D12069002800
:1083100005D02F46002500990020087511E00027A0
:10832000F9E700228021204602F018F9002815D133
:10833000002F15D02168387888627F1C708A401E13
:108340007082708A019B002806980090E9D1002273
:108350004021204602F002F9002808D00320B9E7A6
:1083600028882168C005C00D8862AD1CE6E7202082
:10837000A0670020AEE70220ACE77047034D044C35
:1083800004A002F0EBF9E560FAE700000400FA054A
:1083900000ED00E0486172644661756C745F48618D
:1083A0006E646C65722E0D0A0000000070B586B018
:1083B00014216846FCF7FDFE0F480124418B00297B
:1083C00000D14483408B012805D0022801D100F060
:1083D00001FC06B070BD0122084E950229463046C8
:1083E000FEF729FC00210291039100950194694652
:1083F0003046FEF757FBECE7240100200004005054
:1084000010B505242407002204212046FEF713FCA2
:10841000002208212046FEF70EFC0A2002F003FC91
:10842000012204212046FEF706FC0A2002F0FBFB95
:10843000002204212046FEF7FEFB10BD10B50524E6
:108440002407002204212046FEF7F5FB0122082123
:108450002046FEF7F0FB0A2002F0E5FB0122042192
:108460002046FEF7E8FB0A2002F0DDFB0022042193
:108470002046FEF7E0FB10BDF8B5002405260746B0
:1084800025463607002204213046FEF7D4FB0A2099
:1084900002F0C9FB012204213046FEF7CCFB600646
:1084A000040E08213046FEF7B9FB002801D0641CF9
:1084B000E4B2052002F0B7FB6D1CEDB2082DE1D34C
:1084C000002F03D0FFF79CFF2046F8BDFFF7B6FF53
:1084D000FAE770B505260546360700220421304626
:1084E000FEF7A9FB0024E80901D0012200E00022E8
:1084F00008213046FEF79FFB6806050E0A2002F0B1
:1085000092FB012204213046FEF795FB0A2002F07F
:108510008AFB002204213046FEF78DFB0A2002F080
:1085200082FB641CE4B2082CDDD370BD10B50524B9
:108530002407012208212046FEF77DFB01220421A9
:108540002046FEF778FB002208212046FEF773FB49
:108550000A2002F068FB002204212046FEF76BFB94
:1085600010BD10B505242407002204212046FEF783
:1085700062FB002208212046FEF75DFB0A2002F084
:1085800052FB012204212046FEF755FB012208215F
:108590002046FEF750FB0A2002F045FB10BD70B5E7
:1085A00005252D070024012208212846FEF743FB5C
:1085B000062002F038FB012204212846FEF73BFB8F
:1085C000062002F030FB07E0641CE4B2FA2C03D969
:1085D000FFF7C7FF012070BD08212846FEF71EFBEC
:1085E0000028F1D1002204212846FEF724FB0020B8
:1085F00070BD0000F8B501F023FD01F05DFD5B48A2
:108600000068C069FDF7F4FC594C5A49A082898F73
:10861000594E0025002931D0A26A730357499A4266
:1086200002DB02220A7000E00D700A780121890243
:10863000002A05D0012A0ED0022A10D0032A1DD10B
:10864000608B01282ED0022818D1484808214038D4
:10865000FFF720FC12E0FF22F5329042F0D2608B4F
:1086600001281DD0022804D008E03046FEF7E3FAC6
:1086700004E03E4808214038FFF7CEFBFDF7A2FD9D
:1086800020700121C9023046FEF7C8FA0127FF0316
:1086900000282DD03A480560E079002804D007E092
:1086A0000022E2E70122E0E70120E07101F0B8FFDB
:1086B00080213046FEF7B2FA002806D000220821B9
:1086C0003046FEF7B8FA012205E0012208213046C3
:1086D000FEF7B1FA0022052039460007FEF7ABFA93
:1086E000244C284E4034A08C274F012803D01CE096
:1086F000E5710022EAE725486946088072B68021C4
:108700002348FDF79DFB002804D00222694620483B
:10871000FDF73AFC62B61FA002F020F8A58403F032
:108720005FFF642002F078FAFE60608C012808D1B7
:1087300010486584058003F053FF642002F06CFA52
:10874000FE60208C012806D1258403F049FF6420B7
:1087500002F062FAFE600748124A0188914202D193
:10876000C088002800D1FE60F8BD0000A8160020D7
:1087700024010020DC0D00200004005082000020B5
:10878000680100200400FA0500ED00E0AAAA00003C
:10879000384A0008BDF8C8EBC9FDBCB6C4A3CABDC1
:1087A0000D0A0000AA55000008B55721202000F04E
:1087B0006AF80321212000F066F84021222000F011
:1087C00062F80821232000F05EF8AA21302000F092
:1087D0005AF8084801210187322000F054F802219C
:1087E000332000F050F8684600F006F80A2002F046
:1087F0001AFA08BDDC0D002010B501460F2000F06C
:1088000021F8002800D0012010BD10B50446FFF764
:108810008DFE3220FFF75DFEFFF7C1FEE0B2FFF7ED
:1088200058FEFFF7BCFEFFF781FE3320FFF751FE35
:10883000FFF7B5FE0020FFF71FFE0446FFF791FE8D
:10884000204610BD10B50C46FFF7DFFF2070012059
:1088500010BD70B50D460446FFF768FE3220FFF7E5
:1088600038FEFFF79CFEE0B2FFF733FEFFF797FEFE
:108870002846FFF72EFEFFF792FEFFF772FE0A2052
:1088800002F0D1F970BD10B5FFF7E3FF012010BD74
:1088900010B50248FEF71BFB10BD0000E0150020DC
:1088A000FEB50446002772B6334A01688B1804D11E
:1088B0003248C76803208004074088680190C86870
:1088C000009048698E69002B08D12C4940398B6A89
:1088D000CD042B438B628B6AAB438B6201463143E1
:1088E0003CD025492368CB4205D12449CA680323DB
:1088F0009B049A43CA6025462035002810D0216881
:108900000A6901231A430A61216848610821204647
:1089100000F036F8032800D1A873216808204860C9
:10892000002E10D0206801690122114301612068E6
:1089300086611021204600F023F8032800D1A87397
:108940002168102048600C482168C14206D10B48BC
:10895000C1680322920491433943C16020680169D0
:1089600049084900016121680198886021680098E0
:10897000C86062B6FEBD00000084FFBF4010024028
:1089800070B506460B480D46002409490068FCF7FF
:10899000B1FB7D21C90048433168401E00D103244A
:1089A0000B682A469A4301D00028F6D1204670BDB4
:1089B000204E0000780100201CB5002116480091CF
:1089C000144A01910260C16312054260816007226E
:1089D0008263012202610246C16020321170FF23CE
:1089E0005170C23343628162117301638161042259
:1089F00041634261C161FDF7FFFC084800908013AC
:108A0000019069460448FDF7A7FC00210248FDF7E4
:108A10004DFC1CBD00240140841500200200000410
:108A200008B50848016B012211430163006B012165
:108A30001040009000220A20FEF796FB0A20FEF765
:108A400087FB08BD00100240F0B587B014216846CE
:108A5000FCF7AFFB4748C26A04210A43C262C26AFC
:108A60000A400592C16A80263143C162C16A314021
:108A70000591C16A01242143C162C16A2140059167
:108A8000C16A02252943C162C06A22462840059076
:108A900005201C210007FEF7CEF801223649374891
:108AA000FEF7C9F8002236493448FEF7C4F8912190
:108AB0000520002209020007FEF7BDF831480190A9
:108AC000002705206946029700940007FDF7EAFF9A
:108AD0000C200090112001900320039005200297A4
:108AE00069460007FDF7DEFF10206A46039591C234
:108AF000052069460007FDF7D5FF11200190029778
:108B00006946039700941D48FDF7CCFF1E4801906D
:108B10006946009502941948FDF7C4FFE0020090F1
:108B20006946019702951548FDF7BCFF174869464D
:108B300091C1694611480397FDF7B4FF91200002E7
:108B4000694691C10520694600070397FDF7AAFF12
:108B500069460A48019700960294FDF7A3FF002298
:108B600001210520FEF700FB0520FEF7F1FA07B012
:108B7000F0BD00000010024001020000000400509F
:108B80000830000000001110000021100832000021
:108B900010B50F4C0D482060FF20053060600020AC
:108BA000A060E06020616061E06101212062490213
:108BB0006062A161A0620720E0622046FEF721FF0B
:108BC0002068016840221143016010BD003001405F
:108BD0001016002010B58AB0002404940594069461
:108BE0000794089401211848099400940194029470
:108BF000890703940160092184604160046113497D
:108C00004461C160FEF7C8FF01200003049004A97D
:108C10000D48FEF7EFFF0C48FFF7DEF8089408A9AF
:108C200009480994FEF78CFF6020009008480190E5
:108C300002940822694603940348FFF769F8024842
:108C4000FFF740F80AB010BD68160020930400003A
:108C50005702000000B585B014216846FCF7A9FA58
:108C60000E480D490160E121490241600021816007
:108C7000C160016181610C22C161426101623021E8
:108C800041620121090381634900C163FFF73AFA98
:108C900001F0C0FC05B000BD00380140A81600205E
:108CA00070470000F0B589B00A2002F007FD7D2072
:108CB000C00002F01DFDFF4C0025A570FE48A06518
:108CC000A07B0C2801D30B20A073FC48E570FC4E60
:108CD00000783071FB49A079097840000843217D74
:108CE00089000843F071206BF070010A3172401C5A
:108CF00020636079F449B0744200C81FFE38FCF765
:108D00003FFA6079F04982004000801960311330E9
:108D1000121DFCF735FA607906214200484380199C
:108D2000EA491730921CFCF72BFA2C20205E002811
:108D300003D0E749098A0818A0856079DD49E04E2B
:108D4000C000203182190B7B53764B7B9376062231
:108D50007272E04A1D301278B272A27F32733246CC
:108D6000133A0B781375497851750022314602F099
:108D70008FFD60790021C0001D3002F09BFD0220B4
:108D800002F0ECFCF5712574E57201276773257319
:108D9000D148FEF777F9A0840646E5706079FCF7C4
:108DA000D1FCCE4ACE4BFCF7B1FB01F0D1FE002244
:108DB000BB07FCF7F7FAFCF725FD0006C10C881984
:108DC00080B2F903E084884201D3401AE084C548A8
:108DD00020642079401C2071BF48FEF753F960845D
:108DE000B9484C380390FBE1BB48FEF74BF960846F
:108DF000BD4E0BE0B848FEF745F980B26084E18CC7
:108E0000884203D3B94A8918884206D300210F202B
:108E100002F0D4FB30426063ECD0606B411C21D087
:108E200040047DD58122D20100210F2002F005FDF2
:108E30007D20C00002F05CFC002002F00EFC00214E
:108E4000102002F0BBFB41069F48490E2646002237
:108E50006438616502F0E8FB9B486438417A072971
:108E6000C1D101E001F0F8FC0222A149401DFCF74C
:108E7000ABF90028B7D102F06EFD7166344630665A
:108E800002F056FDF166B066F0786A46401CF0705C
:108E90008D486B38017A1170407A507010880290BA
:108EA000318C88427ED18648924E8C30C08E308084
:108EB00083488C30008FA0838748FEF7E3F86084F6
:108EC00002F08EFAFF22A16E5204E06E0023891890
:108ED00058410206080A1043410849000090080E54
:108EE0000902216760677648636E0A30226E02F0DD
:108EF00007FD6079E36E81007148A26E0818163094
:108F000002F0FEFC6E48636F1230226F02F0F8FC34
:108F10006B4808214172E07C002816D0022200E054
:108F200051E1694872495F38FCF74EF900280CD1CD
:108F300063482774C771606D63491638C2B24E39F1
:108F400008466274EA30FCF71BF960790022800061
:108F50005B491C3002F09CFC6079002180001C30D1
:108F600002F0A8FC009802F0A2FB012002F0F6FB40
:108F7000607202216048FDF751FE00281FD00021D9
:108F800050484F4A01708C324A49508E079088876A
:108F9000908E0590C887E06B1146EC312064086024
:108FA000C43900E0CAE06064C97C8C460907090F37
:108FB000032900D0A174616D1C2902D016E00121A3
:108FC000DEE73F493B4A8C31C98FD1853F4A039B3D
:108FD000083A1B881381884207DD002805DD002937
:108FE00003D0A07D401CA07500E0A5756046000977
:108FF000E074257101202F49E0724031079A0A8000
:10900000059A4A802073A08B3C49FF30C33080B260
:10901000A08388420BD949424018A08330887D2123
:10902000401C80B2C9003080884200D33580368829
:109030007D20C000A18B70434018A0640890304888
:10904000302107782F48E77300884843FCF75FFB1F
:1090500001900A2031464143E08B30220790504373
:10906000081AFCF749FB0199FCF751F97F21C90562
:10907000FCF7B7F8FCF78DFB80B221497F1E088012
:10908000B84201D10120207326851820205EFCF70C
:1090900045FB06460391608CFCF754FB1A4A1B4BB8
:1090A000FCF734FA02900F460898FCF737FB3B4672
:1090B000029A2DE0700000203F420F0024010020A2
:1090C000501200206401002068130020A414002026
:1090D0001C0E002034010020E0150020B81E85EB96
:1090E00051B8CE3FA086010000D02724983A000056
:1090F000480100206001002000040050E703000048
:109100004001002044010020F853E3A59B843E4029
:10911000FCF7EDF93246039BFCF744F9FCF74EFBF4
:10912000E064079800F0C6FC607A002861D1002155
:109130000F2002F043FA0006F9D55AE0FCF740FF91
:10914000614A03211154FF3A60491D3A538E8B87BF
:10915000928ECA87626D1C2A06D15B4B4200AC33EB
:10916000D318039A12885A8086005748584A6038A4
:109170003018928F02805448E16B303830184160CB
:109180005348E36E8C3830181630A26E02F0B8FBEC
:10919000A16DE06B884207DA4B4960398959012992
:1091A00002D1A06502990691474960398A598242E5
:1091B00016DD012A14DD2146002811DD02980884FD
:1091C000022020700CE0324600210F2002F035FB17
:1091D0006079E178401C814202D0002002F03DFA23
:1091E000608CE18C884200D2FEE53A4A89188842B8
:1091F000FAD8E07A012801D00220E07202F0F0F8FB
:10920000354A00210F2002F018FB2079002811D0E8
:10921000324909888A008918814200D22570207C51
:10922000002835D028490C310B7848788A78022BF1
:1092300016D02DE0216CA26D323920468A420DDA1B
:10924000C179264A491CC9B2C171128852008A42AA
:10925000E5D20699018402212170E0E7E571DEE79D
:1092600010280CD0C82813D21D4BC91C1818FBF7A6
:1092700087FF03F0B5F9642001F0CEFCF2E5194D4B
:1092800028684000000E03D1C878FCF740FA286037
:109290000F4D00208C352E4622786179183607E074
:1092A0004300EF5AF35A9F4200D00222401CC0B242
:1092B0008842F5D32270084A002180320F2002F044
:1092C000BCFA09B0F0BD0000F813002070000020C7
:1092D000DC120020983A000000D02724340100203E
:1092E000DC0D00204C01002070470000F0B58BB071
:1092F000002005900A2002F0E1F97D20C00002F074
:10930000F7F9BE4800218170026BBE4C521C02630B
:10931000BB4A838D128A2546D21882854175214623
:1093200013310891203047310390313520461338EE
:10933000B54F02910690B14E0F21B448717100787B
:109340002071B34AB079127840001043327D920008
:109350001043E071308EE070000A2072A174314633
:109360001E2284310898FBF70BFF40222846A949AA
:10937000FBF706FF039902980A7BC274497B0175CB
:1093800009206072A44831460078A072B07F207333
:10939000707D843140004218069910780875507825
:1093A000487576200022974902F072FA70790621FA
:1093B000484300211C3002F07DFA022002F0CEF971
:1093C00000210F2002F0FAF838427063F8D0706B79
:1093D000411C18D040047DD58122D20100210F20EC
:1093E00002F02BFA0021102002F0E8F8410685482F
:1093F000490E0022B43002F017F98248B430417AA5
:10940000022902D0D3E001F027FA02228349401D4D
:10941000FBF7DAFE0028F5D178480222407D4100B2
:109420007648843009187748B530FBF7CDFE002820
:10943000E8D102F090FA714E7166306602F078FA67
:10944000F166B0660598002847D101206D49059066
:1094500073488C31C98E01806A488C30008FB0838C
:109460007048FDF70FFE7084B08B6F49FF30C3303A
:1094700080B2B08388420DD949424018B083684811
:10948000694A01880B32491C89B20180914201D39B
:109490000021018062487D210088C900B28B4143D0
:1094A0008918B16461490A88D1B2F1738C460146CA
:1094B0000A3909B27185002903DA7D23DB00C91856
:1094C00071856146491E8A4201D10121317330857F
:1094D000F08B00E08CE000F0EDFA4A4869468C30F1
:1094E000428E0A80808E488046490422B531C81FCA
:1094F000FF38FBF745FE4148464A407D0099800011
:1095000011503E48FF23816EC06E5B040022C918D3
:10951000504100060E0A0643304602F0C8F87108B2
:1095200049000A0E0802354900264A6708670846BE
:10953000436E026E3348483802F0E2F92F48C36E9A
:10954000826E3048443802F0DBF92C48436F026FDA
:109550002C48403802F0D4F92A49002252393C20E4
:1095600002F096F900213C2002F0A4F9012002F05B
:10957000F5F82249487208468078401C887001211D
:109580000520C9030007FCF72FFD1C48407A00287E
:1095900005D100210F2002F011F80006F9D5802234
:1095A00000210F2002F049F914494E7002E01349DE
:1095B000012048701148417D491CC9B241750F29ED
:1095C00000D2B8E60598002810D10C481849C28B83
:1095D000002A02D00B889A4201D90988C183154913
:1095E000C08B0988401E4843134908800BB0F0BD6A
:1095F000124A00210F2002F020F9D8E77000002065
:109600001C0E00205012002000D02724240100202E
:10961000640100205414002034010020480100207F
:1096200060010020E0150020E70300004001002059
:10963000300100202E0100202C0100200090272462
:10964000F8B531492F48086002F06EFA2F4800F053
:10965000F1F92F4CE0822D48801C00F0EBF92083BB
:109660002A48001D00F0E6F960832B482949418013
:10967000014640310979294F0906090E617006D16A
:10968000C7800121C1870A21418700218187244A9F
:10969000C18E1170C18F6171818FA171817AE1706A
:1096A0008588052165626181C6883046FBF722FD09
:1096B000A08101462846FBF71DFD8800081885B2E9
:1096C000164825816843FCF73DF8164A164BFBF710
:1096D00085FFFCF797F8E081658231463846FBF755
:1096E00009FD20820146C820FBF704FD20840120EB
:1096F000A083FCF77DFCA082E2890C490C48FDF7B1
:10970000C5FCF8BD4DA6000868000020004F000809
:109710002401002026020000DC0D0020E8030000E8
:1097200018000020F853E3A59B843E40FF7F000013
:10973000E0150020F0B5994D85B001202880984FA4
:10974000C820984C3880207A401C2072C00706D070
:10975000E08B411EE183022801D2C820E083E08B28
:1097600000F0A8F90A2001F0A9FF7D20C00001F057
:10977000BFFF02218C48FDF751FA00283FD000209E
:109780008A49800009788B4E490008438849097846
:109790000843B072102070728748C1887D20C000D5
:1097A000FBF7A8FC7073854883490078B073304696
:1097B0000B308A780270C97841707F49421C203191
:1097C0000B7ED370497E11717B49D01C22310B7EF8
:1097D0005371497E9171784940310A7C0271497C0C
:1097E000417100223146172002F052F80021172063
:1097F00002F060F8022001F0B1FF714E03E0012099
:10980000BEE7FEF7F7FE00210F2001F0D7FE304241
:109810006063F6D0606B411C7ED040047DD5812210
:10982000D20100210F2002F008F80021102001F0E1
:10983000C5FE41065F48490E0022B430616501F063
:10984000F3FE5C4EB436707A112866D102225D496F
:10985000701DFBF7B9FC00285FD1F01F027A694642
:109860000A70407A4870B17A2980C820FBF742FC20
:109870003880307BE0833046534D2838C08E2880B6
:1098800030462838008FA0835048FDF7FBFB80B29C
:1098900060840390A08B4E49FF30C33080B2A08318
:1098A00088420CD949424018A08328884849401C66
:1098B00080B20B312880884201D3002028802D8877
:1098C0007D20C000A18B68434018A06402904148ED
:1098D000067828460A3800B2E6736085002803DA65
:1098E0007D21C90040186085388830214843FBF746
:1098F0000EFF07462A20205EFBF7FEFE3946FBF7E7
:1099000006FD7F21C905FBF76CFCFBF742FF3149DF
:1099100080B20880761E01E03EE03BE0B04201D11B
:109920000120207325851820205EFBF7F7FE0746EF
:1099300001910398FBF706FF274A284BFBF7E6FD4A
:1099400005460E460298FBF7E9FE2A463346FBF72A
:10995000CEFD3A46019BFBF725FDFBF72FFFE064A8
:1099600068460088208413481249B430807CC7318F
:109970006071420008460D465130FBF701FC6079EA
:10998000294642001648FBF7FBFBE08BFF2801D07D
:109990000320207005B0F0BD00F05EFF3401002010
:1099A0004401002070000020000400502901002024
:1099B0002A01002050120020DC0D00201800002099
:1099C00000D027244801002060010020E01500207D
:1099D000E703000040010020F853E3A59B843E40CC
:1099E0008013002070B586B014216846FBF7E1FBB8
:1099F00001250F4EED03002229463046FDF71BF9E5
:109A00000120002401900294694600950394304699
:109A1000FDF748F8032001900294694600950394ED
:109A20003046FDF73FF8022001F0F6F806B070BDB1
:109A3000000400500088704770470000F8B50446E5
:109A400000206A461080194D55222A70AA226A7099
:109A50000322AA70661DEE702A716971144A4900CA
:109A60008918AC712246E81DFBF78AFB002007E04D
:109A700029186A468978128889186A461180401C1C
:109A8000B042F5DB611DA81CFCF708F901466846E9
:109A9000018029190078C87168464078087221460B
:109AA0000931024800F0E2FBF8BD00001E1500205D
:109AB000DC0D002010B51B4C228A01E0891AA1831D
:109AC000A18B9142FAD2228C8BB253431B18E383B1
:109AD000132902D14A431018E083E08B3021484318
:109AE000642164304843104960630968401A4B217F
:109AF000090140182063FBF711FE0C4A0C4BFBF7E1
:109B00006DFDFBF75BFE0B49E062884202DD4A42D5
:109B10008018E062002801DA4018E062064909680E
:109B2000486110BD24010020BC000020F853E3A5CB
:109B30009B843E40FF7F0000E0150020034A11682F
:109B4000382389B2994301431160704700300140C6
:109B500010B5FDF77DF810BD10B59AB034216846F8
:109B6000FBF727FB14210DA8FBF723FB1C2112A8F0
:109B7000FBF71FFB1B4801680324E402A143C21446
:109B800089180160FDF7FCFA17480169A1430161DA
:109B900006200090FF200130029001200390102049
:109BA00004900220099040040B90000100240C90C6
:109BB0000A946846FDF712FD0F200D9003200E90C9
:109BC0000F941094012111940DA8FDF7DDFB812065
:109BD0001290032080041890149412A8FDF722FB21
:109BE0001AB010BD007000404010024010480168DB
:109BF000821511430160C1680E4A1140C1600168BD
:109C00000D4A11400160816849084900816001687E
:109C10000122920491430160C168FD221204914324
:109C2000C160002101610649044888607047000056
:109C3000001002400C40FF88F6FFF6FE00500008BE
:109C400000ED00E070B5026801239B07114C124D36
:109C5000984203D0A04201D0A84203D17026B2435B
:109C60004E683243984203D0A04201D0A84204D1AA
:109C700003231B029A43CB681A4380239A430B6940
:109C80001A4302608A68C2620968816201214161E7
:109C900070BD0000000801400014014010B5CB0663
:109CA000DB0E0121046A99408C430462016A9A40E8
:109CB0001143016210BD30B58468FF252D021B02DF
:109CC0001343AC430B432343836030BD826870234E
:109CD0009A430A4307210A438260704730B5026AFB
:109CE000520852000262026A456883697024A343E5
:109CF0009C080B68A40023430224A2438C6845609F
:109D00001443836149684163046230BD30B5026A1F
:109D100010239A430262036A45688269732424020D
:109D2000A2430C6824021443202293438A684560AE
:109D300012011A43846149688163026230BD30B503
:109D4000026AFF2301339A430262026A4568C369CB
:109D50007024A3439C080B68A400234301246402DD
:109D6000A2438C68456024021443C3614968C163FF
:109D7000046230BD30B5026A01231B039A430262BC
:109D8000036A4568C26973242402A2430C68240252
:109D900014430122520393438A68456012031A4315
:109DA000C46149680164026230BD30B5036A046A67
:109DB0006408640004628469F025AC431201224304
:109DC0000A24A3430B438261036230BD30B5036AAA
:109DD0001024A34303628469036A0F252D03120331
:109DE000AC432243A024A3430901194382610162C9
:109DF00030BD0000F8B5102605252D07AE62AF2056
:109E0000800000F010FFFCF791F9364834490068F3
:109E1000FBF740FAFBF7A4FC334CA085AE6101F0E0
:109E2000E1FB324F324EE0650EE001F0DBFBE06516
:109E3000FEF7E0FBA06B411CA163142804D92DA000
:109E400000F08CFC2F48C760E06DB042EDD10026D9
:109E5000A66320780127FF03030000F0B8FC050487
:109E60000C192D303200012239462846FCF7E3FE5A
:109E7000FFF760FC06E0012239462846FCF7DBFECE
:109E8000FFF734FA002239462846FCF7D4FE18E0E2
:109E9000A07A0122401EA07239462846FCF7CBFE6C
:109EA000FCF7C2F8002239462846FCF7C4FEA07A27
:109EB000002806D1267004E0FEF7F4FE01E0FFF76B
:109EC00015FA02211048FCF7A9FE002805D0002051
:109ED0000E49087001F06CFAF8BD0120F8E70000A7
:109EE0000000C84200000020700000200400FA05B5
:109EF0003001CADE4457204944204552524F522E69
:109F00000D0A000000ED00E0000400506401002094
:109F100010B5818CC90707D001684A6801235B042A
:109F20009A43836A1A434A60818C890707D501687E
:109F30004A6801231B049A43C36A1A434A60818C0E
:109F4000490707D501684A6801239B049A43036BBC
:109F50001A434A60818C090707D501684A680123C2
:109F6000DB039A43436B1A434A60818CC90607D5C9
:109F70000268916801231B039943836B1943916025
:109F8000818C890607D501688A6801235B039A439F
:109F9000C36B1A438A60818C490612D503685A68DC
:109FA00001210905046C8A4322435A60026C8A42EB
:109FB00007D10268516803235B059943436C194339
:109FC0005160818C090607D501684A680123DB04CA
:109FD000806C9A4302434A6010BD0000F8B5044605
:109FE000002680300660FCF72DFE054620680068DC
:109FF000124F000709D501212B46002249052046B2
:10A00000009700F0ABFA00280DD1206800684007E7
:10A010000BD501212B46002289052046009700F030
:10A020009DFA002801D00320F8BD2020A067E0673A
:10A030002666603426750020F8BD0000FFFFFF0192
:10A04000F8B5184CC826E078002829D16079002896
:10A0500026D101206071144D686B002700281ED0A6
:10A06000686BC821081A15E01048E168405C616916
:10A0700088470F480A21008848430E490880E06855
:10A08000401CE060E068C82800DBE760696BC8201E
:10A09000401A761EE168814201D0002EE4DC67712F
:10A0A000F8BD00005400002000000240140D002004
:10A0B000340100204601002070B5224CE0780028D1
:10A0C0003FD1207900283CD1012020711E4EF1693A
:10A0D00000250906002933DA2156625791420AD138
:10A0E000F06940062CD5A079002829D0A5712089D7
:10A0F000401C208124E0A179002903D1A0710A200D
:10A1000000F091FD00202056CC2148430F49421811
:10A11000206912181279B262401C00222061A256F6
:10A12000CC235A43895881420ADC25612078401C9F
:10A13000207020780E2800D12570A078401CA070D7
:10A14000257170BD5400002000380140EC01002052
:10A1500010B5806A0022014640314A834A82FDF7E9
:10A16000BFFE10BD70B5846AA06FE56F2168896875
:10A1700000260906002906DA212804D152200653B8
:10A18000204600F06BF820688068400606D5222D36
:10A1900004D15A200653204600F047F8204680306C
:10A1A00001681022114301602046FDF799FE70BD41
:10A1B00010B501460968806A096889061CD4002226
:10A1C0005A210A5201680A68FF2301339A430A6040
:10A1D00001688A68520852008A6001688A684023D0
:10A1E0009A438A602021C167016E012904D1016868
:10A1F0000A6810239A430A60016E012902D0FEF713
:10A2000051F810BD5821095AFDF768FE10BD10B570
:10A21000806A016E012902D0FEF745F810BD582171
:10A22000095A4908FDF75AFE10BD01680A68FF2364
:10A2300021339A430A6001688A68520852008A6092
:10A24000016E012904D101680A6810239A430A604B
:10A250002021C167002101664166704701680A68D4
:10A26000C0239A430A6020218167704770B5164C5D
:10A27000E278002A0CD12279002A09D10122E27069
:10A280000025C82903DC0222A256002A01DCE57061
:10A2900070BD0123E356CC2253430C4AD150012315
:10A2A000E356CC2673439B180A460146181DFAF75D
:10A2B00067FF6078401C607060780E2800D1657080
:10A2C000A078401EA070E2E754000020EC010020BE
:10A2D000F8B50446016880682369E6691843636934
:10A2E000002533431843724A0B68724E33400343D0
:10A2F0000B602168486803231B039843E3681843F5
:10A3000048602168A069914201D0236A18438B6894
:10A310000B263602B34303438B60674923686748C3
:10A320008B420CD1C0688007800F06D0012839D03D
:10A33000022835D0032821D11EE001271FE0604903
:10A340008B420AD1C0680C21084027D0042829D0AC
:10A35000082825D00C2811D10EE093420ED1C168F7
:10A3600003208002014019D001208002091A19D06F
:10A37000091A15D0814201D1082700E010274F4962
:10A38000504840398600934232D1002F0CD0022F22
:10A390000DD0042F10D0082F7FD126E00027EEE744
:10A3A0000227ECE70427EAE7FDF7BCF806E00968B6
:10A3B000C90605D4304603E0FDF7D4F8002872D072
:10A3C000626851005118814267D81103814264D3F9
:10A3D000010E06025008002330185941FAF7A0FE7A
:10A3E00003210902411A384A55E00120C003E7E77A
:10A3F0000122E369D20393422BD13B0000F0E7F93D
:10A400000906090C4D114D4D4D274D00FDF78AF8F9
:10A4100009E0FDF797F806E00968C90605D430465B
:10A4200003E0FDF79FF800283DD0616840004A082E
:10A430008018FAF75FFE80B20146244A1039914233
:10A440002BD8511C01400007400F084329E010465B
:10A45000EBE73B0000F0BBF90906090C21122121B2
:10A4600021232100FDF75EF80AE0FDF76BF807E015
:10A470000968C90606D4304604E00EE0FDF772F81C
:10A48000002810D061684A081018FAF733FE80B22D
:10A4900001460E4A1039914203D9012503E01046C6
:10A4A000F0E72168C86000206066A0662846F8BD15
:10A4B00000480040F369FFEF0038014040100240BF
:10A4C0000044004000093D00FFFC0F00EFFF0000CA
:10A4D000F8B50446416540300026274602838037A0
:10A4E0003E602220E0672546206F603500281CD0A2
:10A4F0001749C162216F17480863216F16484863E6
:10A50000206F8663236F606D9C4613462168024668
:10A5100060462431FCF7EEF9002806D010203860A0
:10A520002E752020A0670120F8BD2E7520680168D7
:10A53000FF2201321143016020688168012211432A
:10A540008160206881684022114381600020F8BD4D
:10A55000B1A100080FA2000865A10008FFB581B0F5
:10A5600005460F46044660350A9E39E0701C37D018
:10A57000FCF768FB0499401AB04222D8002E20D084
:10A580002068016849072BD5C069C043000527D45E
:10A5900001202168C002086220680168FF22A13200
:10A5A000914301602068816849084900816020204A
:10A5B000A067E0678034206000202875032005B084
:10A5C000F0BD20680168FF22A1329143016020683C
:10A5D00081684908490081602020A067E067EBE7B7
:10A5E0002068C1693846884305D00021039881421C
:10A5F000BCD00020E3E70121F8E7000010B50449D2
:10A600001020096808620248FDF76CFC10BD0000CC
:10A61000A816002001490D208870704754000020C2
:10A6200010B507480A22018A51434184FEF7F8F920
:10A63000FEF710FBC82203490348FDF703FE10BDD7
:10A6400024010020140D0020A8160020F8B53E4C6F
:10A65000002321783D4A1D46082910D0072947D0FC
:10A66000062950D0052952D0042953D0032954D0AB
:10A67000002956D0012958D002295AD05BE0A17890
:10A6800000264A1F04E0314FBF5DFB189BB2761CC9
:10A690009642F8DB667927799A195118E37862783F
:10A6A000C9188918C9194018C0430006000E1AD1EC
:10A6B000012E14D0022E16D125482449C018FAF7CD
:10A6C0005FFD01F08DFF642000F0A6FABFF34F8F0D
:10A6D00021492048C860BFF34F8F00BFFDE75908EC
:10A6E0001046FFF7ABF92570E570A570A571F8BDB0
:10A6F000A1795054491CC8B2A071A178491F884261
:10A70000F5D1082001E0607007202070F8BDE070EE
:10A710000620FAE760710520F7E7A070E5700420D5
:10A72000F3E7552807D10120EFE7AA2803D102203B
:10A73000EBE7032803D02570E570A570F8BD032072
:10A7400020702071F8BD00001C010020BA14002008
:10A75000DC0D00200400FA0500ED00E010B5024A0F
:10A76000024900F0E5F910BD19B900087C0100208C
:10A770002021020C01D010211046020A01D01046FF
:10A780000839020901D01046091F820801D010467D
:10A79000891E420801D0881E7047081A7047F8B514
:10A7A000040C8BB2264682B25E430D0C1046370C69
:10A7B0005843360480190021794116466E43370C00
:10A7C00036048019794126466E438919F8BD30B4A4
:10A7D0007446641E2578641CAB4200D21D46635D3E
:10A7E0005B00E31830BC18474900CA02024310005E
:10A7F00000D004204A0D01D001221043044A490D23
:10A80000914201D102210843012800D1052070475F
:10A81000FF0700008307FF22DB0E9A408907090E1D
:10A820009940002808DB830809489B001B1818681A
:10A8300090430843186070470007000F08388308EA
:10A8400004489B001B18D86990430843D86170479F
:10A8500000E400E000ED00E0BFF34F8F044903483F
:10A86000C860BFF34F8F00BFFDE700000400FA058A
:10A8700000ED00E0F8B504464F1EC8000838211866
:10A8800015461E46086849683A4606239A4310D082
:10A890002A463346FAF73AFE3A46D200083AA31857
:10A8A0001A687F1E5B68FAF77DFD06223B469343DC
:10A8B000EED1022F23D0042F11D0062F2FD12A46FC
:10A8C0003346FAF723FEE36AA26AFAF76BFD2A46DB
:10A8D0003346FAF71BFE636A226AFAF763FD2A46DB
:10A8E0003346FAF713FEE369A269FAF75BFD2A46DD
:10A8F0003346FAF70BFE63692269FAF753FD2A46DD
:10A900003346FAF703FEE368A268FAF74BFD2A46DE
:10A910003346FAF7FBFD63682268FAF743FDF8BD9A
:10A92000002210B5134610460149FAF757FE10BD34
:10A930000000F03F10B5FAF735FD10BD002210B54C
:10A94000134610461146FAF749FE10BD10B507210F
:10A95000024A00200907FAF7B9FE10BD0103000002
:10A96000034A10B500201107FAF7B0FE10BD000031
:10A9700001FDFFFF02E008C8121F08C1002AFAD13A
:10A9800070477047002001E001C1121F002AFBD16F
:10A9900070470000014908607047000080010020F6
:10A9A00008B50021684601706B46012202212C2067
:10A9B00000F052FF0221684601706B4601222C20F4
:10A9C00000F04AFF08BD000038B504466D20694616
:10A9D00008706B46012207492E2000F03DFF064912
:10A9E000002C01D0054A00E0054A2E2000F01AFF95
:10A9F00038BD000006080000061800000706000029
:10AA00000716000038B504466B46022200213620A6
:10AA100000F0EEFDB3212300FFF7D9FE0E0F08155D
:10AA20003A3A3A3A1C273A3A2F34483A00216846D3
:10AA3000017040784108490014E0694608788008B0
:10AA40008000401C04E06946087880088000801C73
:10AA500008701DE0684602780A404832027041786A
:10AA6000802001436846417012E0684602780A403F
:10AA7000027040784106490EF4E7694648780221A1
:10AA8000084303E069464878FD210840694648705C
:10AA90006B4601220021362000F0DEFE012200ABD1
:10AAA00011463620013300F0D7FE38BD69460878DC
:10AAB000CF21084069462030CAE708B5032168461F
:10AAC0004170012101706B4602220021362000F006
:10AAD000C3FE0122D20306212D2000F0A3FE012097
:10AAE00000F09AF80120FFF78DFF08BD08B5020AB3
:10AAF00069464A7008706B46022204212D2000F03E
:10AB0000ABFE0320694608706B46012206212D200A
:10AB100000F0A2FE0020694608706B460122062163
:10AB20002D2000F099FE0A212D2000F047FD08BDE0
:10AB3000F8B516460F460446002503E03946B047EF
:10AB4000641C6D1C20780028F8D12846F8BD000050
:10AB5000F8B54A002B4B520DD6182B4A0C46054629
:10AB6000142E2BDA002E12DA284BFAF71BFC0022E7
:10AB70001346FAF78DFE40D2002C03DA0124E407D5
:10AB800000253AE02046284337D0214C14E0214FDD
:10AB90000B46F7403B402B4331D01C4BFAF702FCED
:10ABA00000221346FAF774FE27D2002C03DD0120A1
:10ABB0000005F0400419BC4300251EE0332E1EDCC6
:10ABC00033460027143BFF43DF40384217D00F4B7A
:10ABD000FAF793FC00221346FAF75AFE0DD2002C26
:10ABE0000ADD142E0CD03420811B0120884040192E
:10ABF000A84200D2641C0546BD4321462846F8BD44
:10AC0000641CF9E701FCFFFF9C7500883CE4377E7B
:10AC10000000F03FFFFF0F007D2110B5C900484341
:10AC200000F001F810BD002140E000BF00BF00BFF0
:10AC300000BF00BF00BF00BF00BF00BF00BF00BF1C
:10AC400000BF00BF00BF00BF00BF00BF00BF00BF0C
:10AC500000BF00BF00BF00BF00BF00BF00BF00BFFC
:10AC600000BF00BF00BF00BF00BF00BF00BF00BFEC
:10AC700000BF00BF00BF00BF00BF00BF00BF00BFDC
:10AC800000BF00BF00BF00BF00BF00BF00BF00BFCC
:10AC900000BF00BF00BF00BF00BF00BF00BF00BFBC
:10ACA00000BF00BF00BF00BF00BF491C8142BCD332
:10ACB0007047FFB581B01E460F46040026D00B99A1
:10ACC00003980143A06A394382680720904700280F
:10ACD00018DB0A99A06A3143826806209047002851
:10ACE00010DB25462035A979032F01D9082001431F
:10ACF000032E01D904200143A06A826809209047ED
:10AD0000002806DA0120C04305B0F0BD0020C04392
:10AD1000FAE7384600F000F92060304600F0FCF811
:10AD200060600A9868700398A870EF702E710B9895
:10AD300068710020E8E70000F7B50446002090B0F5
:10AD400000900190002C05D06A46062101F082FC9B
:10AD5000062803DA0020C04313B0F0BD68464078EF
:10AD600001026846007800040918684680780818CF
:10AD7000FAF7E8FC05466846039100790102684647
:10AD8000C07800040918684640790818FAF7DAFC18
:10AD9000032206460F4692075C4BFAF779FD07D26D
:10ADA00000225B4B30463946FAF7A1FB06460F46B8
:10ADB00003229207554B28460399FAF769FD07D2FB
:10ADC0000022534B28460399FAF791FB054603915D
:10ADD0002068FAF7B7FC02460B4630463946FAF7C8
:10ADE000FDFB07460A200791205EFAF797FC3A46DA
:10ADF000079BFAF78BFB064608200991205EFAF7BD
:10AE00007BFC0021C943FAF7C0FAFAF719FD324674
:10AE1000099BFAF7C7FA069108906068FAF792FC66
:10AE200002460B4628460399FAF7D8FB05461A2036
:10AE30000E46205EFAF772FC2A463346FAF766FBA6
:10AE40000C9009911620205EFAF768FC099B0C9A79
:10AE5000FAF7A8FA05910A902A4633463846079928
:10AE6000FAF754FB059B0A9AFAF750FB05910A90F2
:10AE70001420205EFAF752FC3A46079BFAF746FB8D
:10AE800007461C200791205EFAF748FC2A46334605
:10AE9000FAF73CFB0E900B911820205EFAF73EFC6F
:10AEA0000B9B0E9AFAF77EFA2A463346FAF72EFBE8
:10AEB0000B910E902069FAF731FC0B9B0E9AFAF772
:10AEC00071FA2A463346FAF721FB05460E46E0683A
:10AED000FAF724FC2A463346FAF764FA3A46079B07
:10AEE000FAF760FA059B0A9AFAF75CFA01229207D0
:10AEF000084BFAF70BFB02460B46129C0898069982
:10AF000003C411980CC0002026E70000FFFF5F413A
:10AF100000007041E17A843F00B50121C9040300BB
:10AF2000FFF755FC081A05080B0E1114171A032019
:10AF3000C00400BD0720C00400BD0F20C00400BD38
:10AF40001F20400300BD3F20400300BD7F20400381
:10AF500000BDFF20400300BD084600BDFEB5264FE2
:10AF60000D4604000FD0002D0DD0264600202036BF
:10AF7000B071F07129680D208847002801DA780047
:10AF8000FEBD102801D03846FEBDA562E968002943
:10AF900001D028208847204600F030F80028F3DB55
:10AFA000A06AA52182680E209047A06A9621826837
:10AFB0000F209047A06A0221826862209047A06A11
:10AFC000002182680E209047A06A002182680F202D
:10AFD00090477179302001910090062320220121B1
:10AFE0002046FFF766FE0028CEDB204600F0AEF8D4
:10AFF0000028C9DB0020FEBDFFFFFFFF10B586B0B3
:10B00000044614216846FAF7D4F8002C7ED0A06AD2
:10B01000122143686A4610209847122877D1684663
:10B0200000780122010168464078120300090818DF
:10B0300043492081884201DD801A20816846837857
:10B0400040780007000D18186081884201DD801AE1
:10B05000608168460079012201016846C0781205C6
:10B060000003091868464079000908183549E0606E
:10B07000884201DD801AE060684640790007030BD2
:10B080006846807900021B186846C079181820614C
:10B09000884201DD801A20616846417A007A000208
:10B0A000081802B2284801210904A282824201DD67
:10B0B000521AA2826A46D37A927A12029A1812B26D
:10B0C000E282824201DD521AE2826A46537B127B9F
:10B0D00012029A1812B22283824201DD521A22838E
:10B0E0006A46D37B927B12029A1812B26283824222
:10B0F00001DD521A62836A46537C127C12029A184E
:10B1000012B2A283824204DD501A01E00BE008E093
:10B11000A083A06A016828208847002806DA012059
:10B12000C04306B010BD0020C043FAE7C011C007FD
:10B130002034002800D0802060710020F1E700005A
:10B14000FF070000FFFF0700FF7F000010B50400AD
:10B1500009D0A06A0721826808209047002805DAF4
:10B160000120C04310BD0020C04310BD0720203483
:10B170002070002010BD0000FEB5044600200190A4
:10B1800000906079734940000E5A61782578491E15
:10B190007148CFB20163042D77D0072D75D00021FF
:10B1A0000291217801736C49E37901229205896942
:10B1B000002B6CD0914381616748217A4173217AD9
:10B1C00082698907890B0A4382610021042000F00B
:10B1D00034FB324661492E2000F024FB3846FFF74D
:10B1E000F3FB5F4E0522705D810040185D494318F6
:10B1F00007212B2000F030FB5B49029801220B183D
:10B200000B21282000F028FB705D584980000A5867
:10B210000C21282000F011FBE079554980004018EE
:10B22000A1794900425A0221272000F0FBFA514837
:10B230007E00825B0421272000F0F4FAE0790028E8
:10B2400029D0A07804282CD0282069460872202212
:10B250000621272000F0E6FA02AB01222621272052
:10B2600000F0FAFA444938014018E1788900425860
:10B270000821272000F0E1FAA17A601C627A090215
:10B28000114313D016E000E001E0012188E71143EB
:10B29000F608816190E764220621272000F0C2FAB7
:10B2A000E0E71020694608720246D1E7334901728F
:10B2B000090A4172417A007A0A02024320212720BA
:10B2C00000F0B0FA2E4F0C2123203A6800F0B5FAB6
:10B2D000F01982880421232000F0A4FAA079002824
:10B2E0000BD0E0792749012243180021212000F0EA
:10B2F000B3FA03200190012000902A07120F1001D9
:10B300000243607800218007000B0243019800058A
:10B3100002430098400402432079C00640090243DA
:10B320006079C00602431F2000F087FAA078617898
:10B330000123084302040848DB030261E179490361
:10B3400019430A4302610021082000F076FA002028
:10B35000FEBD000088C70008B001002004280000DE
:10B3600030C70008240000204200002038C7000831
:10B3700058C7000864C7000868C7000841100000EB
:10B3800050C700084400002038B50C4607498A8B96
:10B39000002102432C2000F045FA684604706B46F9
:10B3A000012206212C2000F057FA38BDB001002000
:10B3B00010B5FFF7F5FA10BD10B50446042136208C
:10B3C00000F0FCF80121C902002C01D0084300E084
:10B3D000884302460421362000F02FFA10BD0000F9
:10B3E00038B540206946087000210E2000F0E6F8CC
:10B3F0000446002211460E2000F01FFA6B4601227F
:10B4000000210D2000F028FA074A00210F2000F04B
:10B4100014FA00F0EDF9224600210E2000F00DFA9A
:10B4200002480021017338BDF8FF2724D001002015
:10B43000FEB50546042069460870514C0020607531
:10B4400021462031206348710873A0836063A063A4
:10B4500000F0C8F84B4E206002E000F0C3F8206016
:10B46000B042FAD10020FFF7CDFA00F0BBF8464E0B
:10B4700020603078242801D9243806E00621F9F725
:10B4800039FE0622101A40010843020601040A434D
:10B4900001020A430243B260706000211E2000F0E6
:10B4A000CCF900F09FF820606B4601220021242097
:10B4B00000F0D2F91E20FFF719FB86B2300AA07304
:10B4C0000420FFF713FB074600F08CF820603806D5
:10B4D000000E0DD002206946087101AB0122122135
:10B4E0002D2000F0B9F9A08B012109030843A083A6
:10B4F00000F078F820600620FFF7F8FA6060072077
:10B50000FFF7F4FAA060F006C00E207501D11020FC
:10B510002075C0B200F0DCF9E80707D0FFF7CDFADC
:10B52000A08B0121C9020843A0830AE0052136202F
:10B5300000F02EF81549084002460521362000F09B
:10B5400071F90120FFF75EFA0021042000F036F8BF
:10B55000A0610021262000F031F81521890308435D
:10B5600002460021262000F068F90022262136201C
:10B5700000F058F900F036F820600020FEBD000011
:10B58000B00100203001CADE18000020FFFD0000DD
:10B5900038B5094C89B280B26B46022200F028F817
:10B5A000002806D1684640780102684600780818ED
:10B5B00084B2204638BD0000FFFF000038B50024EB
:10B5C000E44389B280B26B46042200F011F80028EF
:10B5D00006D103216846435C2202D418491EFAD5DD
:10B5E000204638BD10B500210846FFF7E7FF10BD23
:10B5F00038B5002909D0402420436C462070C8B2D9
:10B600007F2906D8607002200AE069460870012090
:10B6100006E0802420436C466070C809A0700320B7
:10B62000694600F0B7FF38BD10B5144603460A4618
:10B6300021461120FFF7DCFF10BD10B5034605229F
:10B6400000211520FFF7D4FF10BD10B503460522D9
:10B6500000211720FFF7CCFF10BD38B505460020AC
:10B660006946087000F0C4F8FF2401342246002D1A
:10B6700001D00322120200210D2000F0D3F8002D8A
:10B6800013D06B46012203210F20FFF7B1FF68465C
:10B690000078000709D5FFF7A3FE224600210D2000
:10B6A00000F0C0F80020C04338BD002038BD10B500
:10B6B000024601210A2000F0C0F810BD10B5044672
:10B6C00000211A20FFF77AFF000D22030005120B5C
:10B6D000024300211A2000F0B0F810BD10B5024658
:10B6E00002492E2000F09EF810BD00000418000052
:10B6F000F8B505466B46012203210420FFF778FFC9
:10B700000126114C3607002D0DD02A4600210C20B1
:10B7100000F088F8694608781021084369460870E7
:10B72000A069304307E069460878EF210840694680
:10B730000870A069B0430B46A061012203210420D8
:10B7400000F08AF8F8BD0000B001002010B50246F4
:10B750000021182000F066F810BD0000F8B507467B
:10B76000002568460570B807204C2E4600280ADAE6
:10B770008020694608706B46012200210D2000F0F0
:10B780006BF801202073F8076946087821D006215C
:10B790000843694608706B46012200210D2000F025
:10B7A0005BF803210F20FFF7F3FE8121C900084257
:10B7B00019D04020694608706B46012200210D20F7
:10B7C00000F04AF80020FFF7F7FD00252673ED434F
:10B7D00009E002210843694608706B4601220021F6
:10B7E0000D2000F039F82846F8BD0000D0010020F7
:10B7F0001CB56B46012203210F20FFF7F9FE6846B6
:10B8000000784022C1091040C9014000814208D09F
:10B81000012069460871024601AB03210D2000F0AA
:10B820001BF81CBD08B56B461A70120A5A7089B213
:10B8300080B2022200F010F808BD38B500236C4633
:10B84000E254120A5B1C042BFADB89B280B2234655
:10B85000042200F001F838BD38B58024002909D051
:10B86000C02528436D462870C8B27F2907D8687064
:10B87000022009E0204369460870012004E02043CB
:10B880006870C809A8700320694600F02DFF38BD14
:10B8900010B51446012312189B029A4202D90020C7
:10B8A000C04310BD0B46821E21460920FFF7D4FF7E
:10B8B000002010BD10B5054A8905126901430A43ED
:10B8C00000210820FFF7B9FF002010BDB0010020C3
:10B8D00038B504466B4601220E212B20FFF788FE67
:10B8E00068460078E10640094001C90E01436846F8
:10B8F00001706B4601220E212B20FFF7ADFF38BDF2
:10B9000010B5002142541C06120A22431B0A491C8E
:10B910000429F7DB10BD000013B501231A46694660
:10B920000248FCF7C1FC00981CBD0000A8160020CE
:10B930007CB5002425466846FFF77FFE0420694653
:10B94000220E2D02154322020C5C1443401EF7D533
:10B95000204629467CBD7CB5002425466846FFF775
:10B9600074FE04206946220E2D02154322020C5C4F
:10B970001443401EF7D5204629467CBDFBF770F9DD
:10B98000FEF7EAF8FDF760F841494248002522C079
:10B9900005608561C56140490562C1600838FBF7F3
:10B9A000FBFAFDF73DF8FDF755F9FDF7F1F8FDF766
:10B9B00003F8052601223607D1033046FBF73BF991
:10B9C000FDF73EFEFCF7F0FEFAF744F9FAF7C6F988
:10B9D000FAF794F9FCF7EAFC0721B015FFF7D4FC5D
:10B9E000FFF7E6FC2D4C0A21208A0122484360849F
:10B9F00011033046FBF71FF92648C8222849C830F2
:10BA0000FCF720FC274F284E207900283DD0607895
:10BA100000283AD0FEF7A0F8257120780F280AD91F
:10BA2000012211033046FBF706F9FEF7E3F9002285
:10BA30000121090309E0012251033046FBF7FBF81D
:10BA4000FEF7D8F90022012149033046FBF7F3F84D
:10BA5000FCF7D0FD608C002801D0401E60841348A4
:10BA6000618C00780843CFD13878002801D00328B2
:10BA7000CAD10121C9023046FBF7D0F80028C3D152
:10BA800001210846FBF79CFBBEE7FCF7B3FDBBE7D3
:10BA9000007C0040E0150020FFFF00002401002092
:10BAA000140D002082000020000400505A000020E5
:10BAB00010B586B01748FBF7F2F914216846F9F77C
:10BAC00078FB15480090032001900020029005208B
:10BAD00069460007FAF7E6FF69461048FAF7E2FF01
:10BAE00069460F48FAF7DEFF01210846FBF768FBBD
:10BAF000FF2401342046FBF73BFB0A490868042277
:10BB0000104308602046FBF743FBFBF749FB06B0F8
:10BB100010BD0000E0150020FFFF000000040050F1
:10BB2000000800500070004010B501229202174931
:10BB30001748FAF79FF91548164902888A4223D018
:10BB4000018004218180FF21F531C1800A2101811A
:10BB500000211E224181D24382810122C281818340
:10BB60004323C38602230387782343878287C287C0
:10BB700002464032118451849184C1839180142300
:10BB80008382118200F02CFD10BD0000DC0D00202E
:10BB900000FC0008AA550000F0B51FB496B084461A
:10BBA0000C460246199D18980390490068006300EE
:10BBB000490840080193002A01D0012600E0002630
:10BBC0009E19FE4BF6185B109E422BD36E00039F0E
:10BBD0000296002F00D00127F719F84EF84BBE1936
:10BBE0009E421FD3039E0346F64F334309D03B4684
:10BBF0009C4201D1002A04D0019B002A05D00126D5
:10BC000004E0002039461BB0F0BD00269E19EE4B23
:10BC10009E4207D8039F029E002F00D00127F619ED
:10BC20009E4207D92B4660462146189AFEF782FEAF
:10BC30001BB0F0BD0023002C29DAE44EB04226DA16
:10BC4000E34EB04201DB022321E0DE4EB0421EDBB8
:10BC5000E04E070DBE19142E09DD3427BF1B039ECD
:10BC6000FE400196BE40039FBE420BD00FE0039FF3
:10BC7000002F0CD11427BF1B0646FE400196BE4084
:10BC8000864204D1019BDE07F60F02239B1B0E4662
:10BC9000164318D1002D16DA002C03D0022B01D048
:10BCA000012B06D00220FEF775FEFEF739FE1BB011
:10BCB000F0BD0220FEF76EFEFEF732FE0122D20733
:10BCC00051401BB0F0BD039E002E61D1BF4EB0426B
:10BCD00020D1C148844201D1002A08D0B94881420C
:10BCE00009DB002D10DB189829461BB0F0BD0020A1
:10BCF000B4491BB0F0BD002D06DA01222946D20757
:10BD0000189851401BB0F0BDB4497944086849689F
:10BD10001BB0F0BDAB4FB84225D1002D1FDA002972
:10BD200004D0B14212D1002A09D018E0002A72D101
:10BD3000A649E20F0020D20711431BB0F0BD00203E
:10BD4000E20F0146D20711431BB0F0BDB14206DA43
:10BD5000234600203946F9F741FC1BB0F0BD1046E0
:10BD600021461BB0F0BDB14212DA0126B607B5423A
:10BD700003D1234610461946FEE3994EB54207D13A
:10BD8000261E05DB1046314600F040FC1BB0F0BD1E
:10BD900067007F081646002A40D100290AD08B4A46
:10BDA000914229D1002C0EDD002D1CDB0020114614
:10BDB0001BB0F0BD022B16D0002C14D0012B12D1D9
:10BDC000002C14DB0FE0002C28DA002D09DB012BFE
:10BDD00003D000207D491BB0F0BD002081491BB07D
:10BDE000F0BD012B03D0002001461BB0F0BD0020A8
:10BDF0000121C9071BB0F0BD724A91420ED1002C3F
:10BE000001DA002B17D0022B06D00020C043F9F72F
:10BE100085FC1BB0F0BD90E20120F8E7E217521C50
:10BE200094461A4307D000220892664C62465B1E75
:10BE30001A4307D009E00120FEF7ACFDFEF77EFDB6
:10BE40001BB0F0BD0022644C0892674A90427DDD31
:10BE5000664B674A98421FDD914202DC002D05DBEC
:10BE60004DE05848814217DB002D48DD0220FEF7E7
:10BE700091FDFEF76BFD05460E460022534B214611
:10BE80000898F9F743FB084671004908C00FC0073E
:10BE9000014328461BB0F0BD914215DA002D2EDA81
:10BEA0000220FEF777FDFEF751FD05460E46002203
:10BEB000464B21460898F9F729FB72005208C80F33
:10BEC000C0070243114617E03E4B994223DD002D87
:10BED00015DD0220FEF75EFDFEF738FD05460E4635
:10BEE00000223A4B21460898F9F710FB08467100EA
:10BEF0004908C00FC007014328461BB0F0BD02200F
:10BF0000FEF748FDFEF72CFD49004908E20FD20775
:10BF100011431BB0F0BD002230463946F9F7E7FA6D
:10BF2000012205460E46D243F9F7D0FB314A324B87
:10BF3000F9F7E3FA2A463346F9F7E8FA0022284BE4
:10BF4000F9F7DBFA07462A46334600E064E003913E
:10BF500010461946F9F7DAFA3A46039BF9F7D6FA8A
:10BF60000746032209915207244B28463146F9F728
:10BF7000CDFA07910C90224A204B38460999F9F7DF
:10BF8000C5FA074601911F4A1F4B28463146F9F76B
:10BF9000BDFA3A46019BF9F7AAFA07460B46024654
:10BFA000099107990C98F9F7FDF900250E462846E6
:10BFB000079B0C9AF9F79BFA3A4627E0FFFF1F0010
:10BFC000FFFF0F000000F03F0000E0FF0000F07FE7
:10BFD0000000404301FCFFFF0000F0BF5A0B0000CF
:10BFE0000000E03F0000F0FF0000E0410000F043EF
:10BFF000FFFFEF3F555555555555D53F4715F73F71
:10C00000FE822B6544DF5DF80BAE543E099BF9F7C9
:10C0100074FA02460B4652E1012500202D05A94283
:10C0200007DA352230463946F9F750FB0646342008
:10C03000C0430A151218FE48101803900803FD4962
:10C04000000B01430F46FC49884201DC002003E05D
:10C05000FA49884202DA0120119005E0002011908F
:10C060000398401C7F1B039011980597C200F44869
:10C070000F927844801843680268394630460D9321
:10C080000292F9F734FA07910C9030460D9B029A10
:10C090000599F9F787F902460B460020E549F9F7BB
:10C0A0009DFA09910490079B0C9AF9F72FFA1290C8
:10C0B00000201090E3480D46784400680E9001215E
:10C0C00078104907084311990D9B890440180121F4
:10C0D000C90447183946029A0E98F9F708FA324609
:10C0E000059BF9F70AFA02460B4629461098F9F71C
:10C0F0000DFA064602913B4629460E9A1098F9F72A
:10C1000005FA079B0C9AF9F7F8F93246029BF9F702
:10C11000EEF9099B049AF9F7F9F90591129A0A9038
:10C120002B4610461946F9F7F1F906460246C6486D
:10C130000F460B4606217844FEF79CFB32463B46F1
:10C140000091049010461946F9F7E0F9009B049A13
:10C15000F9F7DCF906460F462B461946129A109855
:10C16000F9F720F9059B0A9AF9F7D0F932463B46D0
:10C17000F9F718F9109A079104902B4610461946C2
:10C18000F9F7C4F9B14E0022334609910290F9F74C
:10C1900009F9079B049AF9F705F9002007460246BA
:10C1A00033460091F9F7A3F9099B029AF9F79FF931
:10C1B000079B049AF9F7A1F906460D913A462946DC
:10C1C000009B1098F9F7A2F907910C902B46304686
:10C1D000129A0D99F9F79AF905460E463A46009BD0
:10C1E00005990A98F9F792F933462A46F9F7DAF8E9
:10C1F00002460B460746099107990C98F9F7D2F8C1
:10C2000000250E462846079B0C9AF9F770F93A4626
:10C21000099BF9F772F907460722099152078C4BDF
:10C2200031462846F9F772F907910090894A884B00
:10C2300038460999F9F76AF907460191864A874B0A
:10C2400031462846F9F762F93A46019BF9F7AAF810
:10C25000834B7B440F9A9B181A685B68F9F7A2F826
:10C26000029009910398F9F759FA05910490099BF6
:10C27000029A07990098F9F795F87A4B7B440F9A40
:10C280009B181A685B6817460393F9F78BF8059BB0
:10C29000049AF9F787F80E462846059B049AF9F7A1
:10C2A00026F93A46039BF9F722F9079B009AF9F71A
:10C2B0001EF9099B029AF9F720F902460B461999D3
:10C2C00000200C900F461898F9F720F9029104907D
:10C2D0003B460C9A19991898F9F709F92A463346FA
:10C2E000F9F714F9029B049AF9F75CF809910E909A
:10C2F0002A46334639460C98F9F708F906460F46A0
:10C30000099B0E9AF9F74EF8574A0D46914220DBE9
:10C310005242AA18024310D132463B46F9F7E7F8D9
:10C3200004900391514A524B09990E98F9F73AF843
:10C33000039B049AF9F7ACFA1ED20220FEF72AFBFF
:10C34000FEF704FB49004908E20FD20711431BB076
:10C35000F0BD6A00474B52089A420DD3464AAA18CC
:10C36000024300D0CBE532463B46F9F7C0F8099BC3
:10C370000E9AF9F78DFAF5D96800002340082C4988
:10C380000393020D3D4B5218984223DD0120000516
:10C39000521CD04042195000400D40183849794491
:10C3A000096813468C463749C1408B43120301216B
:10C3B000120B090551181422101AC1400391002DC7
:10C3C00001DA48420390624630463946F9F78FF861
:10C3D00006460F4632463B4609990E98F8F7E2FFAB
:10C3E00000252A46284B28460591F9F78FF8079132
:10C3F0000C90264A264B28460599F9F787F80091B4
:10C40000029032463B4628460599F9F770F8099B99
:10C410000E9AF9F772F81F4A1F4BF9F777F8009B4D
:10C42000029AF8F7BFFF07460B460246099135E02E
:10C4300001FCFFFF0000F03F8E9803007AB60B006E
:10C440006A070000AC070000D606000000000840A4
:10C4500009C7EE3FFD033ADCF5015B14E02F3EBE59
:10C46000AA0500007005000000009040FE822B65C8
:10C470004715973C00CC904000346F3F0000E03FF0
:10C48000C6040000FFFF0F00432EE63F396CA80CE6
:10C49000615C20BEEF39FAFE422EE63F07990C9808
:10C4A000F8F780FF05460E46079B0C9AF9F71FF830
:10C4B0003A46099BF9F721F809912A4633460E902E
:10C4C00010461946F9F722F8074602462F480B4650
:10C4D000059105217844FEF7CDF93A46059BF9F719
:10C4E00015F82A463346F9F708F807460191284619
:10C4F0003146099B0E9AF9F709F8099B0E9AF8F74D
:10C5000051FF012304910C9000229B0738460199AA
:10C51000F8F7EDFF05910E903A4628463146019B0B
:10C52000F8F7F4FF059B0E9AF9F758F8049B0C9A5C
:10C53000F8F7DDFF2A463346F8F7D9FF0022144BFF
:10C54000F8F7DBFF064603980D460005411909156B
:10C55000002912DC30462946039AF9F7B7F8FEF7AE
:10C5600043F9042801D1FEF7FBF930462946039A26
:10C57000F9F7ACF8064601E004E029180B4632460C
:10C5800021460898F8F7C2FF1BB0F0BD6803000011
:10C590000000F03FF0B58C46002510260521090764
:10C5A0008E620E4C08E067467F5DE760A768FF0774
:10C5B000FCD0E7681F706D1C8542F4DB0020074645
:10C5C00006E0E760A568ED07FCD0E5681D54401C57
:10C5D0009042F6D38E610020F0BD00000030014093
:10C5E00070B572B60124074DA40221462846F9F71A
:10C5F00027FC002804D0224603492846F9F7C4FC4A
:10C6000062B670BD00FC0008DC0D0020F8B50646DF
:10C610000C46F9F74BFA051E0F4600D001200143E6
:10C6200049000B484908411AC90F0DD0002E01D00E
:10C63000012100E000210C4361004908401AC00FAD
:10C6400002D10120FEF7A6F928463946F8BD0000C0
:10C650000000F07FF8B515460E460746002407E0B7
:10C660003819C0B200F008F8641C2870E4B26D1CE0
:10C67000B442F5D33046F8BD10B50446FBF756FF7B
:10C68000EE20FBF726FFFBF78AFF2046FBF721FF92
:10C69000FBF785FFFBF74AFFEF20FBF71AFFFBF7DD
:10C6A0007EFF0020FBF7E8FE0446FBF75AFF20461A
:10C6B00010BD704770B50D460446FBF737FFEE20FE
:10C6C000FBF707FFFBF76BFF2046FBF702FFFBF7CB
:10C6D00066FF2846FBF7FDFEFBF761FFFBF741FF16
:10C6E0000A20FEF7A0FA70BDF0B500251026052738
:10C6F0009C463F070B46BE620C4C06E0595DE1606C
:10C70000A168C907FCD0E1686D1C8542F6DB0020FA
:10C7100007E06146095CE160A168C907FCD0E168F7
:10C72000401C9042F5D3BE610020F0BD00300140B6
:10C730000000010203040005405C0000A05C04004E
:10C74000C06C0800805C0400E03F1E00E07D1E001D
:10C7500007A9022570889B880A00160001000600C0
:10C760000100020087008D002D001A3152001A339B
:10C770009A001A351D011A376B003B31BE003B335E
:10C780005E013B3596023B37000099599959EB51B0
:10C790008F421E45142E0080EB51F5283333E13AC9
:10C7A000703DE13AC235852BC2353333C235C235CF
:10C7B000AE47E13A5138A330513800000000000084
:10C7C00000000102030406070809030406080C1010
:10C7D00018203000000000010203040000000000E7
:10C7E000000000000000F03F000000000000F83FE3
:10C7F00000000000000000000000004003B8E23F1D
:10C80000000000000000000006D0CF43EBFD4C3ECE
:10C81000033333333333E33FFFAB6FDBB66DDB3FC3
:10C820004D268F515555D53F01411DA96074D13F0B
:10C8300065DBC9934A86CD3FEF4E454A287ECA3F05
:10C840003E5555555555C53F93BDBE166CC166BF87
:10C850002CDE25AF6A56113FF16BD2C541BDBBBE80
:10C86000D0A4BE726937663E0000000000000000E0
:10C8700090C800080000002084010000745B0008DC
:10C88000F0C8000884010020541A000084A90008A0
:10C890000124130704380D091E0805400826091055
:10C8A0004008560A131D043B08BE0516D8BC4010AC
:10C8B0000852010338C842035E5C121B0202C51411
:10C8C0000901022281F01F66810498899686967973
:10C8D000821598039814988796749778824397885E
:10C8E000967197778249D90145294B92049220008D
:04000005080050C1DE
:00000001FF
